:20000000020D27021004E4782DF22202100C7845E2FF22021014E47845F22202101C020C02
:20002000A42222021024220100000002102CFFFFFFFFFF021034FFFFFFFFFF02103CFFFFB9
:20004000FFFFFF207F40021044FFFF02104CFFFFFFFFFF021054FFFFFFFFFF02105CFFFF4A
:20006000FFFFFF021064FFFFFFFFFF02106CFFFFFFFFFF021074FFFFFFFFFF02107CFFFF8C
:20008000FFFFFF0210840204A6E59620E7FB75960EE4F597E59620E7FB759691E59620E780
:2000A000FB7814E597F2782CE2B40511E59620E7FBE4F5967823E2F597E4782CF27814E21E
:2000C000FF30E20FE59620E7FB759611E4F597782CF222EF30E41AE59620E7FB7596117514
:2000E0009708E59620E7FB759611759780E4782CF2782CE2600221B47814E220E00221B4C0
:200100007BFE7A0079207D087C007F20120A947823E2FE18E27C0012057A782512057678DF
:20012000271205767820E2547F6421703108E214700221B414601314601A24F9601114603C
:20014000182402706C120BAE806A1200218065120CE38060120022805B1200268056782121
:20016000E2B40C00504B90016C25E0732184218921B1218E21B12193219821B1219D21A26B
:2001800021A721AC1205D8802B12080080261206DD8021120A0A801C12028480171208CF00
:2001A0008012120663800D120A518008120B7A8003120C6D782CE2640170577814E220E1EA
:2001C00051E59620E7FB759691E59620E7FB7814E597F2E230E40320E038781474021205F4
:2001E0009C400B1205A81207C112054A800912058D1207C112056B1205B4B5070818E2B557
:20020000060312056BE59620E7FB7596117814E2F597782CE26402706AE59620E7FB759672
:2002200091E59620E7FB7814E597F2E230E054744012059C400B1205A8120A9412054A806E
:200240000912058D120A9412056B1205B4B5070818E2B5060312056B782CE270127821E273
:20026000B4090C781D120E14120DB6FF120B0B782CE264046005E59620E7FB759611781478
:20028000E2F597227822E224DF7002612F14700261462421B40500400261529002A525E0F1
:2002A000500205837341AF41BB41DA41F161037A0E799512094B900E9580447A0E79A712A7
:2002C000094B900EAAE493FE900EA9E4937C002400782BF2EC3E18F2807B7823E275F00306
:2002E000A42438F8120E14781D120E2D120DB6804E7BFF7A0E79B0781D120E2D900EB0E40E
:2003000093803C7823E2FF64817047EF7BFFB4810E7A0E79C2781D120E2D900EC2800C7ABF
:200320000E79C9781D120E2D900EC9E49380107BFF7A0E79B9781D120E2D900EB9E493FF3A
:20034000E4120957800F7A0E79D01209377426F28003120C6D7822E2FF64016013EF640253
:20036000600EEF64036009EF64046004EFB405177827E2FFD3782BE29F18E2940040087811
:2003800026E27003120952782CE264046008E59620E7FB12092122780074FFF2E47807F212
:2003A000120C662401120C5424FE604314604A24026002816C900113E0FEA3E0FF120C66A2
:2003C0002403F9E43AFAC003C002C001120C4CFD780DE4F208EDF2D001D002D003120971F4
:2003E000120C4CFF900113E48FF0120DE1817078077401F2120C5B8077120C662402F9E4BF
:200400003AFA7818120E2D781B7404F27BFE7A007901120C2678057410F2087401F2780142
:20042000120E08EF2401FFEE3410FEE43DFDE43CFCC004C005C006C0077805E2FE08E2FFBB
:20044000E4F8F9AA06AB07D007D006D005D004C3120DF7501B7805E2FE08E2FF120BFF78F1
:2004600006E22400F218E23402F280B2E47800F29000907461F0A37403F07800E2A3F07B85
:20048000017A0079907847120E2DE92401120C547846F27F611207507807E26008C27FE465
:2004A000F5D712100122C0E0C0F0C083C082C0D075D000C000C001C002C003C004C005C032
:2004C00006C007E59620E7FB759686E59620E7FB7811E597F2E59620E7FB759682E5962028
:2004E000E7FB7812E597F2E59620E7FB759684E59620E7FB7813E597F27811E230E103120F
:200500000D0C7811E230E203120C897812E230E0031200897812E230E1031200067813E27C
:2005200030E10312086D7811E230E003120D15D007D006D005D004D003D002D001D000D002
:20054000D0D082D083D0F0D0E032781FE22440F218E23400F2782BE224C0F218E234FFF21B
:2005600018E22440F218E23400F2227814E24408F2E4782CF222E2FE18E2240008F2EC3E7F
:2005800018F222120E14E92FF9EA3EFA22782AE2FC08E2FD781D120E147F2022F2C3782B5D
:2005A000E2944018E2940022781D120E147D407C007F20227826E2FE08E2FF7829E222E224
:2005C000FD7C0008120E147F2122ECF208EDF24C22D3E29F18E29E227822E2700F08E2700E
:2005E0000B7826E2700608E264026003120C6D7820E2247F6012146028240270537824E22A
:20060000704E08E260138048781CE2B404097824E2700408E2600280377BFF7A00792980B5
:2006200025781CE2B404057824E2600280227825E2B4811A782DE27BFFB403067A0079273A
:2006400080047A0079291209397402F280058000120C6D782CE264046008E59620E7FB12C9
:20066000092122781CE2640260227820E2701D7824E2701808E2701408E2701008E2700C85
:200680007822E2700708E2D394014005120C6D803C7823E2D39400402C781C7404F2E478DF
:2006A0002DF2E59620E7FB12096AE59620E7FB759612759704E59620E7FB75960EE4F59769
:2006C0001200068008781C7403F2782DF2782CE264046008E59620E7FB12094422781CE21C
:2006E000640470567820E2FF60506401604C7822E270477824E270427826E2703D08E260B8
:200700000280377820E2640270307823E2702B7825E2FF64816005EF6402701EEFB4811D9C
:20072000E59620E7FB12096AE59620E7FB759611759710782D7403F28003120C6DE596204B
:20074000E7FB12095E6008E59620E7FB12094422A2AF9200C2AFE59620E7FB75960E7597E2
:2007600001E59620E7FB759691E59620E7FBAF97782DE2FEB4030DE59620E7FB7596117545
:2007800097108038EE7035782D04F2EF30E50BE59620E7FB759611759740EF30E20BE59651
:2007A00020E7FB759611E4F59778461205BF120AD0E59620E7FB759611759701A20092AFA2
:2007C000227815EFF27818120E2D78161205CA602DE59620E7FB7815E2F596E4FFFED3780D
:2007E00017E29F18E29E40167818120583120DB6F597E59620E7FB0FBF00010E80E022FF0D
:20080000781CE2640470507820E2FF604A640160467822E270417824E2703C7826E270378E
:2008200008E2600280317820E26402702A7823E270257825E2FF6481701DEFB4811CE59684
:2008400020E7FB12096AE59620E7FB759611759740E4782DF28003120C6DE59620E7FB1214
:20086000095E6008E59620E7FB12094422E47814F2E59620E7FB75960E759701E59620E724
:20088000FB759694E59620E7FBAF97782DE2B4030CE59620E7FB75961475972022EF30E6C2
:2008A0000BE59620E7FB759614759780120CD278411205BF120A947842120E14120DB6FF14
:2008C000120B0BE59620E7FB759614E4F597227820E26480701B7822E2701608E270120863
:2008E000E2700E08E2700A08E2700608E264016005120C6D801B781CE2FFB4040B7BFF7ACE
:2009000000792712093904F2EFB4030512093304F2782CE264046008E59620E7FB120921EF
:20092000227596117597407401782CF2E47828F208F2227A0079297BFF781D120E2D782A76
:20094000E4F20822759611759748227BFF781D020E2DE2FF08E2CF782AF208EFF222759675
:200960000EE4F597782CE264042275960E75970122780A120E2D7808EEF208EFF2780FEE14
:20098000F208EFF2780DE2FE08E2FF7809E22FFD18E23EFC780FE2FE08E2FFC39DEE9C50E1
:2009A0001D780AE475F001120E1D120DB6FD120BD87810E22401F218E23400F280C622E55C
:2009C0009620E7FB759601759708E59620E7FB759607759707E59620E7FB75960975970719
:2009E000E59620E7FB75960B75970775D7E0E59620E7FB75960F75978043E602D2AFE596DB
:200A000020E7FB759601759701227820E2701B7824E2701608E2701208E2700E08E2700A58
:200A20007822E2700508E230E703120C6D782C7405F27823E2781C60057403F2800374024F
:200A4000F2782CE264046008E59620E7FB12094422781CE2640470227820E26481701B787E
:200A600022E2701608E2701208E2700E08E2700A08E2700608E264016005120C6D8005127E
:200A8000093304F2782CE264046008E59620E7FB120921227815EFF27818120E2D78161208
:200AA00005CA602B7815E2F5964396C0E4FFFE78171205D14016E59620E7FB7818120583F4
:200AC000E597120DCF0FBF00010E80E3E4F596227808EFF2780B120E2D78091205CA602ABE
:200AE000E59620E7FB7808E2F596E4FFFE780A1205D14016780B120583120DB6F597E596F2
:200B000020E7FB0FBF00010E80E3227845E270357842120E14120DB6B4552A78457401F213
:200B20007842120E147818120E2DE92401F9E43AFA120DB6781BF27B017A0079D1120C26ED
:200B4000782F7401F222D27F120C5B7F007E10120CBCBFAA05C27F12100112001ED2AF121F
:200B600009BF120016E4782FF2782FE260FB120397E4782FF212001680EF7820E264017015
:200B80001A7826E2701508E270117822E2700C08E2700808E2700408E26003120C6D782C97
:200BA000E264046008E59620E7FB12094422120CD27842120E14781D120E2D7826120952BA
:200BC000782CE264046010E59620E7FB759611759740740212092922A2AF9200120D1E8E48
:200BE000088F0975B7A575B7F1438F01120D20850982850883EDF0538FFEA20092AF22A2D1
:200C0000AF9200120D1E8E088F0975B7A575B7F1438F03120D20850982850883E4F0538F50
:200C2000FCA20092AF227815120E2DE4FF781BE2FEEFC39E50157818120D02120DB6FE78D2
:200C400015120D02EE120DCF0F80E2227842120E14E92402F9E43AFA020DB69001137410F4
:200C6000F0A37401F0227842120E14E922E59620E7FB75960EE4F597E59620E7FB759611C2
:200C8000759720782C7404F222781C7402F2E59620E7FB759601759701E4782CF20874036D
:200CA000F208F22243B203E4F5B943B980120CF343B9C0120CF3E5B930E5FB22A2AF92008F
:200CC000C2AF8E088F098F828E83E493FFA20092AF227B017A00794E7842120E2D784174E7
:200CE0000AF222782CE264046008E59620E7FB12094422E4FFFE0FBF00010EBE01F8BFF45A
:200D0000F522120E14E92FF9E43AFA227815E22401120564227815E2240112056422C2AF6A
:200D200075FF8075EF0222787FE4F6D8FD75812F75D900020D71020B46E493A3F8E493A31F
:200D40004003F68001F208DFF48029E493A3F85407240CC8C333C4540F4420C8834004F4FA
:200D600056800146F6DFE4800B0102040810204080900E36E47E019360BCA3FF543F30E5E3
:200D800009541FFEE493A360010ECF54C025E060A840B8E493A3FAE493A3F8E493A3C8C59B
:200DA00082C8CAC583CAF0A3C8C582C8CAC583CADFE9DEE780BEBB010689828A83E02250D0
:200DC00002E722BBFE02E32289828A83E49322BB010689828A83F0225002F722BBFE01F393
:200DE00022C5F0F8A3E028F0C5F0F8E582158270021583E038F022EB9FF5F0EA9E42F0E998
:200E00009D42F0E89C45F022E2FC08E2FD08E2FE08E2FF22E2FB08E2FA08E2F922FAE2FBD3
:200E20000808E2F925F0F218E2CA3AF222EBF208EAF208E9F2228830FFFFFFFFFFFFFFFF38
:200E40006040004E00000000000000000000000000000000000000000000000000000000A4
:200E6000000000000000000000000000000000000000000000000000000000000000000072
:200E8000000000008938FF0EF6FF0EFBFF0F27832C00030300120110010000004025130000
:200EA000000000010200010902290001010080AF0904000002030000000921010100012268
:200EC00026000705810340000A0705020340000A0600FF0901A1018555953F750826FF00B6
:200EE00015000901910285619502750826FF00150009018102C005030904002A03610075A7
:200F000000730074007200690061006D006900630072006F00730079007300740065006DEF
:200F2000007300200000002A03410053007800780078002000550053004200200042006F1A
:200F4000006F0074006C006F0061006400650072000000FFFFFFFFFFFFFFFFFFFFFFFFFF44
:200F6000FFFFFFFFFFFFFFFFFFFFFFFFFFFFFFFFFFFFFFFFFFFFFFFFFFFFFFFFFFFFFFFF91
:200F8000FFFFFFFFFFFFFFFFFFFFFFFFFFFFFFFFFFFFFFFFFFFFFFFFFFFFFFFFFFFFFFFF71
:200FA000FFFFFFFFFFFFFFFFFFFFFFFFFFFFFFFFFFFFFFFFFFFFFFFFFFFFFFFFFFFFFFFF51
:200FC000FFFFFFFFFFFFFFFFFFFFFFFFFFFFFFFFFFFFFFFFFFFFFFFFFFFFFFFFFFFFFFFF31
:200FE000FFFFFFFFFFFFFFFFFFFFFFFFFFFFFFFFFFFFFFFFFFFFFFFFFFFFFFFFFFFFFFFF11
:20100000AA02A78702849F900B327402F0E59620E7FB759601759701E4900B42F0A374033D
:20102000F0A3F0220291667814E6FF22028905900A497401F0A37409F0A37415F0900A4899
:20104000740AF022027D9A90087EEBF0A3EAF0A3E9F0A3ECF0A3EDF0A3E07002A3E0700214
:20106000C10F900881E0FEA3E0FF7C007D08129EF090087EE0FBA3E0FAA3E02FF9EA3EFA4B
:2010800090088AEBF0A3EAF0A3E9F0900888E0FEA3E0FF7C007D08129EF0900885E0FBA39E
:2010A000E0FAA3E02FF9EA3EFA90088DEBF0A3EAF0A3E9F0900881E0FEA3E0FF7C007D0816
:2010C000129EF0900890ECF0A3EDF0900888E0FEA3E0FF7C007D08129EF0900892ECF0A322
:2010E000EDF0900890E0FEA3E0FF6D7002EE6C600241ECEF4E7002410E90088AE0FBA3E441
:2011000075F001129F3CA9F0FA129E3CFF900892E0FCA3E0FD244EF582740B3CF583E05F1D
:20112000900898F0C374089DFFE49CFEC3900884E09FEE6480F8900883E064809890088D72
:20114000E0FB403CA3E0FAA3E0F9129E3CFF900892A3E02445F582740B3CF583E05F129EA5
:2011600077900892E0FEA3E0FFC374089FFFE49EFEC3900884E09FF0900883E09EF0807248
:20118000A3E0FAA3E0F9129E3CFF900883E0FCA3E0FD900892E0F8A3E02DFDE83CFC744F62
:2011A0002DF582740B3CF583E0FE900892E0FCA3E02445F582740B3CF583E04E5F129E772A
:2011C000900898E0FF900883E0FCA3E0FD900893E02DFD900892E03CFC74452DF582740B36
:2011E0003CF583E0FEEF5E900898F0E4900883F0A3F090088DE0FBA3E475F001129F3CA9EB
:20120000F0FA129E3CFF900898E04F129E77900883E0FAA3E0FB7C007D08FFAE02129EF0B0
:20122000900894EEF0A3EFF07C007D08AF03AE02129EF0A3ECF0A3EDF0900894E07002A3FF
:20124000E0603F900894E0FEA3E0FF90088DE0FBA3E0FAA3E0F8AC02AD0390088AE0FBA38D
:20126000E0FAA3E0F9129DF4900894E0FEA3E0FF90088BEE8FF0129F2690088EEE8FF012DD
:201280009F26900896E0FEA3E0FF4E7002C10F90088DE0FBA3E0FAA3E0F9129E3CFD744EC7
:2012A0002FF582740B3EF583E05D129E7790088DE0FBA3E0FAA3E0F9C003C002C001129E00
:2012C0003CFF90088AE0FBA3E0FAA3E0F9129E3CFE900896E0FCA3E02445F582740B3CF5D6
:2012E00083E05E4FD001D002D003C10C900892E0FEA3E0FFD3900891E09FEE6480F8900834
:2013000090E06480984070A3E09FFF900890E09E900894F0A3EFF0900894E0FEA3E0FFC37D
:2013200074089F900897F0E49E900896F090088AE0FBA3E475F001129F3CA9F0FA129E3C7D
:20134000FDA807088002C333D8FC90089CF0E0FF90088AE0FBA3E0FAA3E0F9129E3CFE901A
:201360000896A3E0FDEEA805088002C313D8FC4FFF90089CF0804A900890E0FEA3E0FFC3F9
:20138000900893E09FFF900892E09E900896F0A3EFF0900896E0FEA3E0FFC374089F900858
:2013A00095F0E49E900894F090088AE0FBA3E0FAA3E0F9129E3CFDA807088002C313D8FC48
:2013C000FF900892E0FCA3E0244EF582740B3CF583E05F90089CF0900892E0FEA3E0FFC3B9
:2013E00074089FFFE49EFEC3900884E09FEE6480F8900883E064809890088DE0FB403EA393
:20140000E0FAA3E0F9129E3CFF900892E0FCA3E02445F582740B3CF583E05F129E779008F1
:2014200092E0FEA3E0FFC374089FFFE49EFEC3900884E09FF0900883E09EF08072A3E0FA17
:20144000A3E0F9129E3CFF900883E0FCA3E0FD900892E0F8A3E02DFDE83CFC744F2DF58278
:20146000740B3CF583E0FE900892E0FCA3E02445F582740B3CF583E04E5F129E7790089CD7
:20148000E0FF900883E0FCA3E0FD900893E02DFD900892E03CFC74452DF582740B3CF583EF
:2014A000E0FEEF5E90089CF0E4900883F0A3F090088DE0FBA3E475F001129F3CA9F0FA12DC
:2014C0009E3CFF90089CE04F129E77900883E0FEA3E0FF7C007D08129EF0900898EEF0A3DC
:2014E000EFF090089874FFF5F0129F26C364809480406590088AE0FBA3E475F001129F3C77
:20150000A9F0FA129E3CFF900894A3E0FEEFA806088002C333D8FC90089CF0E0FF90088A8A
:20152000E0FBA3E0FAA3E0F9129E3CFE900896A3E0FDEEA805088002C313D8FC4FFF90088A
:201540009CF090088DE0FBA3E475F001129F3CA9F0FAEF129E77808A900883E0FEA3E0FFF7
:201560007C007D08129EF090089AECF0A3EDF04C7002C10F90088AE0FBA3E475F001129F13
:201580003CA9F0FA129E3CFF900894A3E0FEEFA806088002C333D8FC90089CF0E0FF900858
:2015A0008AE0FBA3E0FAA3E0F9129E3CFE900896A3E0FDEEA805088002C313D8FC4FFF9088
:2015C000089CF090089AE0FCA3E0FD2445F582740B3CF583E05F90089CF090088DE0FBA3D0
:2015E000E0FAA3E0F9129E3CFF744E2DF582740B3CF583E05F129E7790088DE0FBA3E0FA2E
:20160000A3E0F9129E3CFF90089CE04F129E7722900B77EBF0A3EAF0A3E9F0A3EDF0E0FE73
:201620005407900B7CF0EEC394085002E18EE4900B7BF0900B7AE0131313541FFFA3E0C36A
:201640009F4002E18E900B77E0FBA3E0FAA3E0F9900B7BE0FF75F008A4F582E92582F9EA64
:2016600035F0FA129E3C9008CAF0900B77A3E0FAA3E0F975F008EFA42401F582E435F0F568
:2016800083E92582F9EA3583FA129E3C9008CBF0900B77A3E0FAA3E0F9900B7BE075F008F5
:2016A000A42402F582E435F0F583E92582F9EA3583FA129E3C9008CCF0900B77A3E0FAA3D1
:2016C000E0F975F008EFA42403F582E435F0F583E92582F9EA3583FA129E3C9008CDF0901C
:2016E0000B77A3E0FAA3E0F9900B7BE075F008A42404F582E435F0F583E92582F9EA35831D
:20170000FA129E3C9008CEF0900B77A3E0FAA3E0F975F008EFA42405F582E435F0F583E978
:201720002582F9EA3583FA129E3C9008CFF0900B77A3E0FAA3E0F9900B7BE075F008A424F4
:2017400006F582E435F0F583E92582F9EA3583FA129E3C9008D0F0900B77A3E0FAA3E0F917
:2017600075F008EFA42407F582E435F0F583E92582F9EA3583FA129E3C9008D1F07BFF7AE8
:20178000A8798E123000900B7BE004F0C133900B7CE0D39400404B900B7AE0131313541FF0
:2017A00075F008A4A3F0900B7AE0FFA3E0FEC39F5027900B77E0FBA3E0FAA3E02EF9E43A05
:2017C000FA129E3C9008CAF07BFF7AA879B7123000900B7BE004F080CD7BFF7AA879BD12A8
:2017E000300022E59620E7FB75960EE4F597E59620E7FB759611759720900B427404F02265
:20180000E4FFFEFDFC90087012A106900870E0F8A3E0F9A3E0FAA3E0FB900A0BE0FFE4FC72
:20182000FDFEEB2FFFEE3AFEED39FDEC38FC90087012A106900870E0F8A3E0F9A3E0FAA3EE
:20184000E0FBC000900A0CE0FFE4FCFDFE780812A0F3D000EB2FFFEA3EFEE93DFDE83CFC16
:2018600090087012A106900870E0F8A3E0F9A3E0FAA3E0FBC000900A0DE0FFE4FCFDFE78B7
:201880001012A0F3D000EB2FFFEA3EFEE93DFDE83CFC90087012A106900A0AE024FE700268
:2018A000214524FE7002219F24FC7002416C24F8700241C5147002614424F170028128241C
:2018C0001F6002A166900870E0FCA3E0FDA3E0FEA3E0FF90088312A1067F16121D9F90084A
:2018E0006F748BF01247EF90086FE0241BF0E0FF126C77900874EFF09008877401F0A374D2
:2019000008F0A3746EF07B017A08796DE4FFFE12580090086DE0540FC3940E400A90086F2D
:20192000E06480946C40C0129B9590086DE0FE540F900959F0EEC4540FA3F090086EE0905B
:20194000095BF0A16E900870E0FCA3E0FDA3E0FEA3E0FF90088312A1067F16121D9F7F0106
:2019600012864512775D90086BEEF0A3EFF0128097900869EEF0A3EFF0E4FF12864590085F
:201980006BE0FAA3E0FF900869A3E0C39F900959F0EAFD900869E0C39D90095AF0A16E900E
:2019A000000FE004F0900861E004F090000FE0FBD3943540097435F0E4900959A16B900805
:2019C00070E0FCA3E0FDA3E0FEA3E0FF75F004EBA4240CF582E5F03400F58312A106900AC5
:2019E0000EE0FF74E32BF582E43400F583EFF0900A0FE0900862F0900870E0FCA3E0FDA318
:201A0000E0FEA3E0FF90000BE0F8A3E0F9A3E0FAA3E0FBC312A0CF5014900870E0FCA3E06D
:201A2000FDA3E0FEA3E0FF90000B12A106900870E0FCA3E0FDA3E0FEA3E0FF90085DE0F81E
:201A4000A3E0F9A3E0FAA3E0FBD312A0CF4014900870E0FCA3E0FDA3E0FEA3E0FF90085D0B
:201A600012A10690095974FCF0A3613F90000F7401F0900861F0900870E0FCA3E0FDA3E044
:201A8000FEA3E0FF90001012A106900A0EE09000E4F0900870E0FCA3E0FDA3E0FEA3E0FF1A
:201AA00090000B12A106900870E0FCA3E0FDA3E0FEA3E0FF90085D12A10690095974FEF069
:201AC000A304F0A16E900A0BE0FF7E00900855EEF0A3EFF0FD900A0CE0FFED900855CFF0F6
:201AE000A3EFF0900A0DE0FF900824EEF0A3EFF0FD900A0EE0FFED900824CFF0A3EFF090C4
:201B00000A0FE0FF900846EEF0A3EFF0FD900A10E0FFED900846CFF0A3EFF090095974FE99
:201B2000F0C3900825E09432900824E09400500CE4F0A37432F090095974FFF090095A743A
:201B4000FFF0A16EE4FFFEFDFC90087412A10674FFFFFEFDFC90087812A10690095974FE52
:201B6000F0A304F0900862E090095BF0900855E0FCA3E090095CF0ECA3F0900824E0FCA335
:201B8000E090095EF0ECA3F0900846E0FCA3E0900960F0ECA3F090085DE0FCA3E0FDA3E086
:201BA000FEA3E0FF900962EFF090085DA3A3A3E0780812A0E0900963EFF090085DE0FCA3AC
:201BC000E0FDA3E0FEA3E0FF781012A0E0900964EFF090000BE0FCA3E0FDA3E0FEA3E0FF35
:201BE000900965EFF090000BA3A3A3E0780812A0E0900966EFF090000BE0FCA3E0FDA3E03A
:201C0000FEA3E0FF781012A0E0900967EFF0900861E0900968F09000E4E0900969F09000AB
:201C20000FE090096AF0A16E900A0FE0FE900A0EE0FDEDFF900874EEF0A3EFF07F07129720
:201C400044900876EFF07F08129744900877EFF0E4FD7F07129916E4FD7F08129916900808
:201C600070E0FCA3E0FDA3E0FEA3E0FF90088312A1067F16121D9F9009577442F0A3744071
:201C8000F0900A5EE0FBA3E0FAA3E02401F9E43AFA129E3C900A5DF0A37401F0A37409F060
:201CA000A37457F090095974FEF0A304F01298BC900874E0FEA3E0FFD394E8EE9403401BDA
:201CC000EF2420FFE43EFEEF7806CEC313CE13D8F9FF7C007D30129E89801A900874E0FE0A
:201CE000A3E0FF7C007D30129E89EF7806CEC313CE13D8F9FF90084BEEF0A3EFF0E490087F
:201D00004EF07F011286457F017E001287DF129A0A129CC67F8F129A75900A10E0B4010515
:201D200012840F80057F9E129A757D0A7C007F807E001291BAE4F50EF50F1299BBEF6006B8
:201D4000121027EF60CEE4FF128645900876E0FD7F07129916900877E0FD7F081299169067
:201D600008547401F02290095974FFF0A3F09009577442F0A37440F0900A5EE0FBA3E0FA6B
:201D8000A3E02401F9E43AFA129E3C900A5DF0A37401F0A37409F0A37457F01298BC229029
:201DA0000882EFF0A3E0FCA3E0FDA3E0FEA3E0FF900B0212A106E4FF12974490088AEFF091
:201DC00054FEFDE4FF129916900882E0641670757B017A0879877D037F161293EE900889F0
:201DE000E0547024F0602024D0602724F0602E24F0603524F0603C2470704390088B740156
:201E0000F0A374F4F0803E90088BE4F0A374FAF0803390088BE4F0A374C8F0802890088BDD
:201E2000E4F0A37464F0801D90088BE4F0A37432F0801290088BE4F0A37419F08007E490F2
:201E4000088BF0A3F090088BE0FEA3E0FBAA06E4F9F8900883E0FCA3E0FDA3E0FEA3E0FFEE
:201E600012A02790089312A106900893E0FCA3E0FDA3E0FEA3E0FF780612A0E0EE543FFE8C
:201E800090088DEEF0A3EFF090088DE0FCA3E0FDAE047806C333CE33CED8F92DFFEC3EFE22
:201EA00090088FF0A3EFF0E4FCFD900893E0F8A3E0F9A3E0FAA3E0FBD312A0CF401C9008EA
:201EC00090E02441F090088FE03400F090088EE004F0700690088DE004F0900893A3A3E058
:201EE000FEA3E0FFC3900890E09FF090088FE09EF090088DE0FEA3E0FBAA06C3900890E077
:201F0000942190088FE09400401C90088EE024FFF090088DE034FFF0900890E024DFF09049
:201F2000088FE034FFF0C3900890E0942090088FE094004011EB1B70011AA3E024E0F09004
:201F4000088FE034FFF090088FE0FEA3E0FFC39420EE940050A5EF9410EE94004010E02409
:201F6000E0F090088FE034FFF0EB1B70011A90088FE0FEA3E0FFC390088EE09FFF90088DC3
:201F8000E09E900891F0A3EFF0900890E02BFF90088FE03AAD07FC900882E064167047EDED
:201FA000AE047806CEC313CE13D8F9540FFF900889E054F04FF0900891E0FAA3E0FBEA54F6
:201FC00003FFAE05EE25E025E054FC4F900888F0900887EBF07B017A0879879008B77403E7
:201FE000F07F16128DAE12700090088AE0FDE4FF029916E4900869F0A3F053C97F029ABAA1
:20200000E4900863F0900866F0A374C8F053D9BF121FF3D2AF1296537BFF7AA679851230CF
:20202000007F5E7EC67D0D7C0090001012A1069000E474D8F07F527EC87D0D7C00900014AF
:2020400012A1069000E574D8F07F467ECA7D0D7C0090001812A1069000E674D8F07F3A7EB9
:20206000CC7D0D7C0090001C12A1069000E774D8F07F2E7ECE7D0D7C0090002012A106907E
:2020800000E874D8F07F227ED07D0D7C0090002412A1069000E974D8F07F167ED27D0D7C1A
:2020A0000090002812A1069000EA74D8F07F0A7ED47D0D7C0090002C12A1069000EB74D8DC
:2020C000F07FFE7ED57D0D7C0090003012A1069000EC74D8F07FF27ED77D0D7C0090003479
:2020E00012A1069000ED74D8F07FE67ED97D0D7C0090003812A1069000EE74D8F07FDA7E9A
:20210000DB7D0D7C0090003C12A1069000EF74D8F07FCE7EDD7D0D7C0090004012A10690D7
:2021200000F074D8F07FC27EDF7D0D7C0090004412A1069000F174D8F07FB67EE17D0D7CEB
:202140000090004812A1069000F274D8F07FAA7EE37D0D7C0090004C12A1069000F374D83C
:20216000F07F9E7EE57D0D7C0090005012A1069000F474D8F07F927EE77D0D7C0090005430
:2021800012A1069000F574D8F07F867EE97D0D7C0090005812A1069000F674D8F07F7A7E79
:2021A000EB7D0D7C0090005C12A1069000F774D8F07F6E7EED7D0D7C0090006012A106902F
:2021C00000F874D8F07F627EEF7D0D7C0090006412A1069000F974D8F07F567EF17D0D7CBB
:2021E0000090006812A1069000FA74D8F07F4A7EF37D0D7C0090006C12A1069000FB74D89C
:20220000F07F3E7EF57D0D7C0090007012A1069000FC74D8F07F327EF77D0D7C00900074E7
:2022200012A1069000FD74D8F07F267EF97D0D7C0090007812A1069000FE74D8F07F1A7E58
:20224000FB7D0D7C0090007C12A1069000FF74D8F07F0E7EFD7D0D7C0090008012A1069086
:20226000010074D8F07F027EFF7D0D7C0090008412A10690010174D8F07F5C7E797D0C7CAB
:202280000090008812A10690010274D8F07FEA7E027D0E7C0090008C12A10690010374D8F9
:2022A000F07FDE7E047D0E7C0090009012A10690010474D8F07FD27E067D0E7C009000949E
:2022C00012A10690010574D8F07FC67E087D0E7C0090009812A10690010674D8F07FBA7E36
:2022E0000A7D0E7C0090009C12A10690010774D8F07FAE7E0C7D0E7C009000A012A10690DD
:20230000010874D8F07FA27E0E7D0E7C009000A412A10690010974D8F07F967E107D0E7C57
:20232000009000A812A10690010A74D8F07F8A7E127D0E7C009000AC12A10690010B74D858
:20234000F07F7E7E147D0E7C009000B012A10690010C74D8F07F727E167D0E7C009000B455
:2023600012A10690010D74D8F07F667E187D0E7C009000B812A10690010E74D8F07F5A7E15
:202380001A7D0E7C009000BC12A10690010F74D8F07F4E7E1C7D0E7C009000C012A1069034
:2023A000011074D8F07F427E1E7D0E7C009000C412A10690011174D8F07F367E207D0E7C27
:2023C000009000C812A10690011274D8F07F2A7E227D0E7C009000CC12A10690011374D8B8
:2023E000F07F1E7E247D0E7C009000D012A10690011474D8F07F127E267D0E7C009000D40D
:2024000012A10690011574D8F090000F7432F01297077F017E001287DF900010E0FCA3E0C7
:20242000FDA3E0FEA3E0FF123800900864EEF0A3EFF04E60177FE87E031287DF900864A332
:20244000E0FF1267687FE87E031287DF7BFF7AA679CB900864E0FFA3E09008CACFF0A3EF6D
:20246000F0123000129C5C7DAA7F007E10129862129C1F900866E07002A3E06010900867D1
:20248000E024FFF0900866E034FFF0803B900864E07002A3E07F0060027F0474C07E5DA8A1
:2024A00007088005C333CE33CED8F9900867F0EE900866F0900868E06006E4F0C2A2800821
:2024C0009008687401F0D2A2126A4980A6E59620E7FB75960EE4F597E59620E7FB75969119
:2024E000E59620E7FB9008C6E597F0900B42E0B40513E59620E7FBE4F596900B39E0F597E0
:20250000E4900B42F09008C6E0FF30E210E59620E7FB759611E4F597900B42F022EF30E4B0
:202520001BE59620E7FB759611759708E59620E7FB759611759780E4900B42F0900B42E040
:202540006002C12A9008C6E020E002C12A7B017A0B79367D087C007F20128F3A900B39E024
:20256000FE900B38E07C002400FFEC3EF0A3EFF0900B3BE0FE900B3AE02400FFEC3EF0A326
:20258000EFF0900B3DE0FE900B3CE02400FFEC3EF0A3EFF0900B36E0547F64217035A3E0FF
:2025A00024FE601B14602224FA600F14601614601D240A7072129479807012950F806B126E
:2025C00037FF8066129B818061124FFE805C124FFF8057900B37E0B40C00504B9025E22595
:2025E000E073A1FAA1FFC127C104C127C109C10EC127C113C118C11DC12212752C802B1259
:20260000875A80261285BA802112920E801C12598F801712888380121286D0800D128CCF51
:20262000800812969180031217E3900B42E064016002C1FA9008C6E030E102C1FAE5962064
:20264000E7FB759691E59620E7FB9008C6E597F0E030E40530E002C1FA9008C67402F0C368
:20266000900B41E09440900B40E09400403C900B33E0FBA3E0FAA3E0F97D407C007F201273
:20268000910F900B34E475F040129F26900B41E024C0F0900B40E034FFF0900B3FE02440DF
:2026A000F0900B3EE03400F08024900B40E0FCA3E0FD900B33E0FBA3E0FAA3E0F97F20121F
:2026C000910F9008C6E04408F0E4900B42F0900B3CE0FEA3E0FFA3E0B50611A3E0B5070C5E
:2026E0009008C6E04408F0E4900B42F0E59620E7FB7596119008C6E0F597900B42E0640229
:202700006002E1DAE59620E7FB759691E59620E7FB9008C6E597F0E020E002E1DA7440F0FB
:20272000C3900B41E09440900B40E09400403C900B33E0FBA3E0FAA3E0F97D407C007F2001
:20274000128F3A900B34E475F040129F26900B41E024C0F0900B40E034FFF0900B3FE02423
:2027600040F0900B3EE03400F0801C900B40E0FCA3E0FD900B337F20128F329008C6E044B7
:2027800008F0E4900B42F0900B3CE0FEA3E0FFA3E0B50611A3E0B5070C9008C6E04408F045
:2027A000E4900B42F0900B42E07019900B37E0B40912900B33E0FBA3E0FAA3E0F9129E3C13
:2027C000FF129000900B42E064046005E59620E7FB7596119008C6E0F5972290086CEBF06A
:2027E000A3EAF0A3E9F0E4FF90086CE0FBA3E0FAA3E02FF9E43AFA129E3C60030F80E922F5
:2028000090087CEBF0A3EAF0A3E9F0A3E0FBA3E0FAA3E0F9129F52FDACF0AE047803CEC3FF
:2028200013CE13D8F9FF900882EEF0A3EFF0ED5407A3F0E92407F9E43AFA12A11290088578
:20284000EBF0A3EAF0A3E9F0E4A3F0A3F0A3F0A3F0A3F0A3F0A37429F075088F90087FE01B
:20286000FBA3E0FAA3E0240AF9E43AFA129E3CF50990087FA3E0FAA3E02402F9E43AFA12D4
:202880009F52FDACF0AE047803CEC313CE13D8F9900889F0ED54076003E004F07E007F2C72
:2028A0007D007B007A00793012A335900882E0FCA3E0FDEC540FC454F0FBED54F0FFE4C473
:2028C000F854F0C8EFC4540F484B7830F6E0540FC4F8540FC868FF7831A607900888740230
:2028E000F0900884E0601625E0540E440146F6900883E004F07006900882E004F0E49008BF
:202900008AF0900883E024FEFF900882E034FFFE90088AE0C39FE49E503390087FE0FBA3F8
:20292000E0FAA3E02404F9E43AFA12A11290088AE0FF29F9E43AFA129E3CFE900888E02FE8
:202940002430F8A60690088AE004F080B590088AE0FF900888E02FF0900884E0FF70024186
:202960003A900888E0FE242FF9C374089FFF74FFA807088002C333D8FC57F7742F2EF8C0A9
:2029800000E6FE90087CE0FBA3E0FAA3E02425F9E43AFA129E3CFD900884E0FCEDA8040888
:2029A0008002C313D8FC4ED000F6900888E0FE2430F8C000E6FD90087CE0FBA3E0FAA3E0FB
:2029C0002425F9E43AFA129E3CFCA807088002C333D8FC4DD000F674302EF8C000E6FF90A0
:2029E000087CE0FBA3E0FAA3E02426F9E43AFA129E3CFE900884E0FDEEA805088002C3133F
:202A0000D8FC4FD000F6900888E02431F8C000E6FF90087CE0FBA3E0FAA3E02426F9E43A8B
:202A2000FA129E3CFEC374089DFDEEA805088002C333D8FC4FD000F6803890087CE0FBA38B
:202A4000E0FAA3E02425F9E43AFA129E3CFF900888E0FE2430F8A60790087CE0FBA3E0FA71
:202A6000A3E02426F9E43AFA129E3CFF74312EF8A607900888E02402F07F071297449008F4
:202A80008CEFF090087FE0FBA3E0FAA3E0240BF9E43AFA129E3CFD7F0712991690087FE072
:202AA000FBA3E0FAA3E0240BF9E43AFA129E3CB4FF047D3E80027D3F7F0D129916E4F50E0B
:202AC000F50F7F8F129A7590087FE0FBA3E0FAA3E02402F9E43AFA129F52FD7F1B1299163F
:202AE00090087FE0FBA3E0FAA3E02402F9E43AFA129F52E5F05403FD7F1A1299169008A0EF
:202B0000741DF0A3E4F0A37400F0A37430F0900888E09008A4F07B007A0079097D01128FBD
:202B2000927F807E00129831E4F50EF50F7F8F129A75E4900888F090087FE0FBA3E0FAA38B
:202B4000E02402F9E43AFA129F5245F0700281837F5E7E80129831E50F30E35C90088DA3CF
:202B6000E0FD7F1B12991690088DE05403FD7F1A1299167F527E001298317F1C129744EFC9
:202B8000540FFFC3940340027F03900885E0FBA3E0FAA3E0F9128C627F8F129A757D3F7F5A
:202BA0000D129916900885E0FBA3E0FAA3E0F9129E3C4480FF029E77E50E30E74290088B21
:202BC0007412F0E50E30E73790088BE0FFB4122F900885E0FBA3E0FAA3E0F9128C629008BE
:202BE0008BE0FFFD900886E48DF0129F26900888E02FF0530E7F7F5E7E8012983180C47FA0
:202C00005E7E00129831E50F541F60207F1C129744EF541FFF90087FE0FBA3E0FAA3E02417
:202C20000CF9E43AFAEF129E777F0822E4F50EF50F7F1C129744EF541FFF90088BF0900839
:202C400088E0FEFDEF2DFDE433FCA3E0FFFBD3ED9B7480F86C984006EF9E90088BF090089F
:202C60008BE0FF900885E0FBA3E0FAA3E0F9128C6290088BE0FF900888E02FF0900889E0D7
:202C800024FEF090088CE0FD7F07129916900888E0FF90087FE0FBA3E0FAA3E0240CF9E4DC
:202CA0003AFAEF129E777D3F7F0D1299167F002290087DEBF0A3EAF0A3E9F0A3EDF0E49043
:202CC0000890F0900887F0A3F0900885F0A3F07FC0FE1298317F5F7E00129831E50F541F74
:202CE000600890089074FFF0E1BF530F7F90088A748FF0A3749DF07B017A08798A7D021215
:202D00009B277D407F1A1299167D3F7F0D1299167F807E001298317F8F129A75E4F50EF56E
:202D20000F7F1BFE129831E50F5417600890089074FEF0E1BFE50F20E302E1BF90087DE092
:202D4000FBA3E0FAA3E02402F9E43AFA7F01128C6290087DE0FBA3E0FAA3E02402F9E43A94
:202D6000FA129E3C54F81313543FFF7E00900883EEF0A3EFF0D39420EE9400400990088303
:202D8000E4F0A37420F0900883A3E0FF90087DE0FBA3E0FAA3E02424F9E43AFAEF129E773C
:202DA000900884E02404F0900883E03400F0E0FEA3E0FF900887EEF0A3EFF07803C333CEC2
:202DC00033CED8F9FF900883EEF0A3EFF0900883E0FCA3E0FDEC5403444090088AF0EDA3C7
:202DE000F0900883E0FEA3E07803CEC313CE13D8F9F0EE900883F07B017A08798A9008B75D
:202E00007402F07F1A128DAEE4F50EF50F90087DE0FBA3E0FAA3E02403F9E43AFA90088D2E
:202E2000EBF0A3EAF0A3E9F0900884E024FF805FC3900884E09412900883E09400405A7FB3
:202E4000067E80129831E50F5407600890089074FDF0E1BF7F1C129744900882EFF0530ED1
:202E60007F90088DE0FBA3E0FAA3E0F97F12128C62900886E02412F0900885E03400F09074
:202E8000088EE475F012129F26900884E024EEF0900883E034FFF08097E4900881F0E50F56
:202EA000545F7066900882E02403F00000E02403F00000E02403F07F1C129744EF541F9010
:202EC0000882F0D39401403690088DE0FBA3E0FAA3E0F97F01128C62900886E004F07006B9
:202EE000900885E004F090088EE475F001129F26900884E024FFF0900883E034FFF09008D5
:202F000081E004F0E0D394C840947F5F7E00129831E50F5415700790088904F08005E49060
:202F20000889F0E4F50EF50F900880E0FF129A757F1C129744EF541F900882F06031E0FFA9
:202F4000FDC3900884E09DF0900883E09400F090088DE0FBA3E0FAA3E0F9128C6290088296
:202F6000E0FF900886E02FF0900885E03400F07F8F129A757F0F12974490087DE0FBA3E017
:202F8000FAA3E02427F9E43AFAEF129E77900889E060069008907401F0900888E024FFF03B
:202FA000900887E034FFF0900885E0FEA3E0FFA3E06E7003A3E06F602490089074FCF0E42C
:202FC000F50EF50F90088A748FF0900880E090088BF07B017A08798A7D02129B27E4FD7F16
:202FE0001A129916900890E0FF2212629F1298BC900A0A7402F0900959E06003B401EB2253
:203000009008C7EBF0A3EAF0A3E9F0E49008F2F0A3F0A3F0A3F0A3F0A3F0A3F0A3F0900882
:20302000FEF0A3F0A3F0A3F0A3F090090A04F0A37408F0A374CAF09008C7E0FBA3E0FAA385
:20304000E0F9129E3C7002813012A13233EB0A308F2533873033AD3133AD3233AD3333AD97
:203060003433AD3533AD3633AD3733AD3833AD3930E24430E25530DA5830E26330E264306F
:20308000AF6830E26C30E27530E27800003401E4900908F0A3F09008F6E07004A3E0640183
:2030A0009008F67007F0A3F07F258110E461969008F6E07002A3E06010900909E004F070BF
:2030C00006900908E004F081139008C7E0FBA3E0FAA3E0F9129E3CFF8110900900E4F0A322
:2030E00004F0E49008FAF0A3F0A3F0A3F09008F6E07004A3E064016002616B90090DF0A38C
:203100007404F0900908E0FEA3E0FF64024E702690090DF0A37402F090090AE0FBA3E475E3
:20312000F001129F3CA9F0FA129E3CFD9008F4E4F0A3EDF08021EF64014E90090AE0FBA3F1
:20314000E475F002129F3CA9F0FA129F52FF9008F4E5F0F0A3EFF090090DE0FFA3E090082F
:20316000F2CFF0A3EFF0D39008F3E094009008F2E094005002418990090DA3E01425E025C9
:20318000E0FD740F7E00A805088005C333CE33CED8F9FF9008F4E05EFEA3E05FA8050880A3
:2031A00005CEC313CE13D8F9FF9008F2E0FCA3E0FD2402F58274093CF583EFF074022DF58A
:2031C0008274093CF583E0FFC3940A402BEFD3940F5025900900E07002A3E07E5760027E94
:2031E00037EE2FFF9008F2E0FCA3E02402F58274093CF583EFF080219008F2E0FEA3E0FF5B
:203200002402F58274093EF583E02430FD74022FF58274093EF583EDF09008F2E0FEA3E096
:203220002402F58274093EF583E0B4302A9008FAE07002A3E070109008FDE004F07026905A
:2032400008FCE004F0801E9008FBE004F070169008FAE004F0800E9008FBE004F0700690AA
:2032600008FAE004F09008F5E0C4F8540FC868F09008F4E0C454F048F09008F3E024FFF0A2
:203280009008F2E034FFF0216690090DE0FEA3E0FF2403F58274093EF583E4F09008F6F0F1
:2032A000A3F09008FEE07002A3E070089008FEEEF0A3EFF09008FAE0FEA3E0FFC39008FF56
:2032C000E09F9008FEE09E4070E49008F2F0A3F09008FAE0FEA3E0FFC39008FFE09FFF9060
:2032E00008FEE09EFEC39008F3E09F9008F2E09E50157F301293099008F3E004F070D19085
:2033000008F2E004F080C99008FAE0FFA3E09008F2CFF0A3EFF09008F2E0FEA3E0FFD39486
:2033200000EE940040571292FD9008F3E024FFF09008F2E034FFF080DD9008FAE0FFA3E077
:203340009008F2CFF0A3EFF09008F2E0FEA3E0FFD39400EE940040251292FD9008F3E0243A
:20336000FFF09008F2E034FFF080DD9008C7E0FBA3E0FAA3E0F9129E3CFF129309E490082C
:20338000FEF0A3F0A380519008F6E07004A3E0640170099008F8F0A304F080779008C7E0A8
:2033A000FBA3E0FAA3E0F9129E3CFF80639008F8E07004A3E064019008C77021E0FBA3E031
:2033C000FAA3E0F9129E3C24D0FEE434FF9008FEF0A3CEF0E49008F8F0A3F08036E0FBA370
:2033E000E0FAA3E0F9129E3CFF80257F0D1293099008C7E0FBA3E0FAA3E0F9129E3CFF800F
:203400000F9008C7E0FBA3E0FAA3E0F9129E3CFF1293099008C7E0FBA3E0FAA3E02401F979
:20342000E43AFA9008C7EBF0A3EAF0A3E9F001372290087EEBF0A3EAF0A3E9F0A3EDF0E499
:2034400090088BF0A3F0A3F0A3F0900891F0A37403F0E4F50EF50F7F8F129A75E490089156
:20346000F0900881E0FF900891E0C39F504D90087EE0FBA3E0FAA3E0F9900891E0FF75F005
:2034800028A4F582E92582F9EA35F0FAE4F5F0129F7DEF75F028A4FF90087EE0FBA3E0FAD3
:2034A000A3E02FF9EA35F0FAE92424F9E43AFAE4129E77900891E004F080A6E4F50EF50FFD
:2034C00090088AE0600F900882E0FBA3E0FAA3E0F9A3E080077B007A007900E4FD125000D2
:2034E0007F2C7E01129C66E4F50EF50F900886E0FF128987E490088DF0A3F07F01FEFDFC81
:20350000900886E0F9F812A0F390088FEEF0A3EFF0900881E0FD90088BE0FEA3E0FFC39DB7
:20352000EE94004002C10D7C007D28129E8990087EE0FBA3E0FAA3E02FF9EA3EFA128E6B59
:20354000EF1460142402706790088EE004F0705F90088DE004F08057900885E0FF7E00C024
:2035600006C00790088BE0FEA3E0FF7C007D28129E8990087EE0FBA3E0FAA3E02FF9EA3E60
:20358000FAE92404F9E43AA801FCAD03900882E0FBA3E0FAA3E0F9D007D00612A311EF70F4
:2035A0000E90088CE004F0700690088BE004F0900890E024FFF090088FE034FFF0E4F50E6C
:2035C000F50F900887A3E0FAA3E0F912A158900893EFF0900881E0FFC390088CE09F9008C4
:2035E0008BE09400501590088FE07002A3E0600B900893E060057F99129A7590088FE070E0
:2036000002A3E06008900893E06002A111900892E014F090088DE07002A3E0607DE47F0155
:20362000FEFDFC900886E0F9F812A0F3E47B04FAF9F812A027A804A905AA06AB0790088DF7
:20364000E0FEA3E0FFE4FCFDD312A0CF500A900886E004F07F9A803DE47F01FEFDFC9008C4
:2036600086E0F9F812A0F3E47B08FAF9F812A027A804A905AA06AB0790088DE0FEA3E0FFE2
:20368000E4FCFDD312A0CF400A900886E014F07F9C80027F9B129A758005E4900892F090C2
:2036A0000881E0FFC390088CE09F90088BE094005017900892E06011900887A3E0FAA3E0A4
:2036C000F912A158EF600281F490088BE07002A3E07021900B0DE024FFF0900B0CE034FF42
:2036E000F0E07002A3E07015FF128645129C2D1244AE8000900B0CE4F0A3740AF090088B96
:20370000E0FEA3E0FF229008A6EBF0A3EAF0A3E9F0A3EDF0E4FFA3E0FBA3E0FAA3E0F91229
:203720009E3CFE9008A6E0FBA3E0FAA3E02402F9E43AFAEE129E779008AAE0FBA3E0FAA30F
:20374000E02401F9E43AFA129E3CFE9008A6E0FBA3E0FAA3E02403F9E43AFAEE129E779073
:2037600008A9E0FEEFC39E50329008ADE0FBA3E0FAA3E02FF9E43AFA129E3CFE9008A6E080
:20378000FBA3E0FAA3E02404F9E43AFAEF7C0029F9EC3AFAEE129E770F80C49008A9E0FFC0
:2037A0009008A6E0FBA3E0FAA3E02424F9E43AFAEF129E779008B0E0FBA3E0FAA3E0F91253
:2037C0009E3CFF9008A6E0FBA3E0FAA3E02425F9E43AFAEF129E779008B0E0FBA3E0FAA344
:2037E000E02401F9E43AFA129E3CFF9008A6E0FBA3E0FAA3E02426F9E43AFAEF029E77222C
:2038000090086912A10690086D7455F0A374AAF0E4A3F0A374FFF07B017A08796D9008B7CF
:203820007404F07F16128DAE7E007F047D007B017A08796D12A3357B017A08796D7D047F0E
:20384000161293EE90086DE0FFB4550EA3E0B4AA09A3E07005A3E0F460257BFF7AA379884E
:203860009008CAEFF090086EE09008CBF090086FE09008CCF0900870E09008CDF02152C221
:20388000A17F017E001287DFD2A17F0C7E001287DF7B017A08796D7D047F161293EE9008F8
:2038A0006DE06455600FA3E064AA6009A3E06005A3E0B4FF087BFF7AA379A82152E4F50E61
:2038C000F50F7D207F0D1299167D027F1E1299167F8F129A757F92129A757B017A08796DD8
:2038E0009008B77404F07F1F128DAE7B017A08796D9008B77404F07F1F128DAE7B017A08A2
:20390000796D9008B77404F07F1F128DAE7B017A08796D9008B77404F07F1F128DAE7B011D
:203920007A08796D9008B77404F07F1F128DAE7B017A08796D9008B77404F07F1F128DAEF7
:203940007F207E00129831E50F20E50E7BFF7AA379B71230007E007F0122E4F50EF50F1242
:203960009C2D7F84129A75129CCCEF24C8601C24E8602614602324FC601F24257023E49071
:203980000AF2F07BFF7AA379DB8024900AF27401F07BFF7AA379F18016900AF27402F080B2
:2039A00016129CCC9008CAEFF07BFF7AA479071230007E007F0F227D02E4FF1299167D0608
:2039C0007F011299167DF07F021299167D0C7F0A12991690086F7460F090086E74D8F09087
:2039E000086D744FF07B017A08796D9008B77403F07F16128DAE7D027F0B12991690086D54
:203A00007401F07403F0A3745DF0A37420F07B017A08796D9008B77403F07F15128DAE7F55
:203A20000B12974490086DEFF04460F0FD7F0B1299167D377F0D12991690086D7403F0A3BE
:203A40007484F0A3740AF07A08796D128DA4E490086DF0A3F0A3F07B017A08796D9008B790
:203A60007403F07F12128DAEE4FF129776900869E0FCA3E0FDA3E0FEA3E0FF90088312A1D1
:203A8000067F16121D9F7FB4126C777F147E001287DF7F0E12974490086DEFF020E0057E2B
:203AA000007F022290086DE020E1057E007F0322E4FEFF22900B70EEF0A3EFF0A3EBF0A3C7
:203AC000EAF0A3E9F0E4FFA3F0A3F0FEFD900B71E024F0900B70E034D8C364809480400F8B
:203AE000A3E024F0F0900B70E034D8F00F80DE900B71E02418900B70E034FCC364809480ED
:203B00004014A3E02418F0900B70E034FCF0900B75E004F080D9900B71E0249C900B70E0C3
:203B200034FFC3648094804014A3E0249CF0900B70E034FFF0900B76E004F080D9900B71B8
:203B4000E024F6900B70E034FFC364809480400FA3E024F6F0900B70E034FFF00E80DE90AC
:203B60000B71E024FF900B70E034FFC364809480400FA3E024FFF0900B70E034FFF00D806D
:203B8000DEEF7002810C2430FF900B72E0FBA3E0FAA3E0F9EF129E77900B75E02430FF903C
:203BA0000B72E0FBA3E0FAA3E02401F9E43AFAEF129E77900B76E02430FF900B72E0FBA392
:203BC000E0FAA3E02402F9E43AFAEF129E77EE2430FF900B72E0FBA3E0FAA3E02403F9E40E
:203BE0003AFAEF129E77ED2430FF900B72E0FBA3E0FAA3E02404F9E43AFAEF129E77900B69
:203C000072E0FBA3E0FAA3E02405A13E900B75E0606B2430FF900B72E0FBA3E0FAA3E0F960
:203C2000EF129E77900B76E02430FF900B72E0FBA3E0FAA3E02401F9E43AFAEF129E77EE08
:203C40002430FF900B72E0FBA3E0FAA3E02402F9E43AFAEF129E77ED2430FF900B72E0FBB4
:203C6000A3E0FAA3E02403F9E43AFAEF129E77900B72E0FBA3E0FAA3E02404A13E900B76F6
:203C8000E060502430FF900B72E0FBA3E0FAA3E0F9EF129E77EE2430FF900B72E0FBA3E09E
:203CA000FAA3E02401F9E43AFAEF129E77ED2430FF900B72E0FBA3E0FAA3E02402F9E43AD6
:203CC000FAEF129E77900B72E0FBA3E0FAA3E02403806BEE60382430FF900B72E0FBA3E096
:203CE000FAA3E0F9EF129E77ED2430FF900B72E0FBA3E0FAA3E02401F9E43AFAEF129E77C4
:203D0000900B72E0FBA3E0FAA3E024028030ED60112430FF900B72E0FBA3E0FAA3E0F9EF64
:203D2000800D900B72E0FBA3E0FAA3E0F97430129E77900B72E0FBA3E0FAA3E02401F9E460
:203D40003AFAE4129E772290086FEBF0A3EAF0A3E9F0AB05900874E0FA75F010A42421FE35
:203D6000E435F0900878F0A3CEF0A3E4F0A37429F0E4A3F0A3F075088F7509917830F60867
:203D800076550876C2AF03EFC4333354C0FF08F6900873E0FE1313543F4FF6EEC4333354E9
:203DA000C0FF08F6EA1313543F4FF6A3E0C4333354C0FF08F690086FE0FBA3E0FAA3E0249A
:203DC00025F9E43AFA129E3CFE1313543F4FF6EEC4333354C0FF08F690086FE0FBA3E0FA3D
:203DE000A3E02426F9E43AFA129E3CFE1313543F4FF6EEC4333354C008F67D3F7F0D1299E0
:203E000016E4F50EF50F7F8F129A75900878A3E0FD7F1B129916900878E05403FD7F1A1298
:203E200099169008A0741DF0A3E4F0A37400F0A37430F0A37408F07B007A0079097D01124F
:203E40008F927F807E00129831E4F50EF50F7F8F129A757F5F7E80129831E50F30E355902C
:203E6000087AA3E0FD7F1B12991690087AE05403FD7F1A1299167F527E001298317F1C126E
:203E80009744EF540FFFC3940340027F03900875E0FBA3E0FAA3E0F9128C627F8F129A75C8
:203EA000900875E0FBA3E0FAA3E0F9129E3C4480FF029E77E50E30E77590087D7412F0E56C
:203EC0000E30E76A90087DE0FF6412706190087CE0FDFBEF2BFBE433FA900874E0FC75F0B9
:203EE00002A4FFD3EB9FE5F06480F8EA6480984009EC25E0C39D90087DF090087DE0FF9086
:203F00000875E0FBA3E0FAA3E0F9128C6290087DE0FFFD900876E48DF0129F2690087CE025
:203F20002FF0530E7F7F5E7E8012983180917F5F7E00129831E50F541F600F7F1C12974426
:203F4000EF541F90087DF07F0822E4F50EF50F7F1C129744EF541FFF90087DF090087CE084
:203F6000FD2FFBE433FA900874E0FC75F002A4FFD3EB9FE5F06480F8EA6480984009EC2549
:203F8000E0C39D90087DF090087DE0FF900875E0FBA3E0FAA3E0F9128C6290087DE0FF9083
:203FA000087CE02FF0900874E075F002A4FF90087CE0B50707E4B5F003FF80027F0822908B
:203FC00008C7EBF0A3EAF0A3E9F0E4FF9008CDE0FEEFC39E50299008C7E0FBA3E0FAA3E015
:203FE0002FF9E43AFA129E3CFE9008CAE0FBA3E0FAA3E02FF9E43AFAEE129E770F80CD2287
:20400000900898EBF0A3EAF0A3E9F0E49008A5F0530F7F7F8F129A757F9D129A757D407F02
:204020001A1299167D3F7F0D1299167F807E001298317F8F129A75E4F50EF50F7F1BFE1280
:204040009831E50F54176002212DE50F20E302415B7B017A0B790E7F01128C62900B0EE062
:2040600054F81313543FFF7E0090089CEEF0A3EFF0D39420EE9400400990089CE4F0A374B9
:2040800020F090089CA3E0FF900898E0FBA3E0FAA3E02424F9E43AFAEF129E7790089DE0CB
:2040A0002404F090089CE03400F0E0FEA3E07803C333CE33CED8F9F0EE90089CF0E0FCA3BD
:2040C000E0FDEC5403444090089FF0EDA3F090089CE0FEA3E07803CEC313CE13D8F9F0EE51
:2040E00090089CF07B017A08799F9008B77402F07F1A128DAEE4F50EF50F7B019008A20446
:20410000F0A3740BF0A3740FF090089DE024FF8051C390089DE0941290089CE09400404CCC
:204120007F067E80129831E50F540660089008A574FFF0415B7F1C12974490089BEFF05342
:204140000E7F9008A2E0FBA3E0FAA3E0F97F12128C629008A3E475F012129F2690089DE0B1
:2041600024EEF090089CE034FFF080A57F407E00129831E50F5415700790089E04F0800546
:20418000E490089EF07F9F129A757F1C129744EF541F90089BF0601FE0FFFDC390089DE096
:2041A0009DF090089CE09400F09008A2E0FBA3E0FAA3E0F9128C627D377F0D1299167F80CC
:2041C0007E001298317F8F129A757D207F1B129916E4F50EF50F7F5FFE1298317F1C129779
:2041E00044EF541FFF60747B017A0B7930128C62900898E0FBA3E0FAA3E02424F9E43AFA38
:20420000129E3CFD9008AA7401F0A3740BF0A3740EF0A37401F0A3740BF0A37410F0A3749F
:2042200001F0A3740BF0A37430F0900898A3E0FAA3E0F91237067F0F129744900898E0FB46
:20424000A3E0FAA3E02427F9E43AFAEF129E7790089EE060069008A57401F0E4FD7F1A1242
:2042600099169008A5E0FF2290086BEBF0A3EAF0A3E9F0A3EDF0E4900874F0900887740A7D
:20428000F0A37432F0E4FD7F1A1299167D507F1B129916128A04C292D293129CDC90086FA8
:2042A000E0FFA3E0FBA3E0FAA3E0F9A3E0900890F0126E81124A1D900885EFF0706C7B013F
:2042C00090089004F0A37408F0A3747DF0A37408F0125C8B90086BE0FBA3E0FAA3E0242401
:2042E000F9E43AFA7408129E7790086BE0FBA3E0FAA3E02404F9E43AFA9008CAEBF0A3EA29
:20430000F0A3E9F090086BA3E0FAA3E02424F9E43AFA129E3C9008CDF07B017A0879751296
:204320003FBF9008747401F0819F900885E0B4FD07E4900874F0819F90088974FFF0A3749E
:204340009CF0A374E6F09008867402F090086EE07002819F900887E0FF900886E0C39F404A
:2043600002819F900888E0FF14F0EF7002819F128A04C292D293900889A3E0FAA3E0F91212
:20438000A158124A1D900885EFF06011240370028141240260028157900889818C9008902D
:2043A0007401F0A37408F0A3747DF0A37408F07B01125C8B900874E075F028A4FFAEF09037
:2043C000086BE0FBA3E0FAA3E02FF9EA3EFAE92424F9E43AFA7408129E7790086BE0FBA3DF
:2043E000E0FAA3E02FF9EA3EFAE92404F9E43AFA9008CAEBF0A3EAF0A3E9F090086BA3E038
:20440000FAA3E02FF9EA3EFAE92424F9E43AFA129E3C9008CDF07B017A087975123FBF90C6
:204420000874E004F090086EE014F0900886E014F090088974FFF0A3749CF0A374E1F061D0
:204440004C90088974FFF0A3749CF0A374E1F0900886E014F0614C900889E0FBA3E0FAA336
:20446000E0F9EB8A8389827BFF7A9C79D7F4700A74D765827004749C6583900889600D7472
:20448000FFF0A3749CF0A374D7F0614C74FFF0A3749CF0A374E6F0900886E004F0614C90DD
:2044A0000874E07003129C2D900874E0FF227B017A0B7906900894EBF0A3EAF0A3E9F024A1
:2044C00002F9E43AFA129E3C9008A0F0900B0B7401F078067C0BFD900894E0FBA3E0FAA381
:2044E000E0F97E007F05129DF49008A0E0D394034002E4F0900B07E07005900B0904F09087
:204500000894E0FBA3E0FAA3E0F9129E3C7002C14524FA7002A1FC24FE7002A1C1146067C9
:2045200024FD602924FD6002C1E2E4900897F0A374C0F0A374F2F0A3744DF0A37401F0A3E9
:204540007404F0A37402F0A37407F0C16BE4900897F0A374C0F0A374C2F0900B0AE0700D1B
:20456000A3F090089A74FAF0E4A3F0800A90089A749AF0A37402F090089C7406F0A3740425
:20458000F0A37427F0C16BE4900897F0A374C0F0A37492F0900B0AE0700EA3F090089A7432
:2045A00038F0A37401F0800A90089A7441F0A37403F090089C7405F0A314F0A37437F0C11D
:2045C0006BE4900897F0A374C0F0A37482F0900B0AE0700EA3F090089A7477F0A37401F072
:2045E000800A90089A74E8F0A37403F090089C7406F0A37404F0A3743BF0806FE4900897BC
:20460000F0A374C0F0A37462F0900B0AE0B4010FE4A3F090089A74F4F0A37401F0800A900E
:20462000089A7435F0A37405F090089C7407F0A304F0900B07E090089E700574BFF0802B02
:20464000743FF08026E4900897F0A374C2F0A37402F0A374D0F0A37407F0A3741BF0A3741E
:204660000FF0A374FFF0E4900B0BF0900B07E025E025E0FF900897E054F34FF054FCFF90BC
:204680000B0AE04F900897F0A3E054FCFF9008A0E04F900898F0900B09E07F0060027F0179
:2046A000EF25E0FF900899E054FD4FF07B017A0879979008B77404F07F01128DAE7F05123E
:2046C0009744EF54F0FF90089BE04FFD7F051299167B017A08799C9008B77403F07F0712C8
:2046E0008DAE22124800900869EFF06002E1B4126926900822E07002A3E07008900869740F
:2047000009F0E1B4128B75900869EFF06002E1B4900A0AE024FE602224FA6052146064242E
:20472000086002E1B4900858E0FBA3E0FAA3E0F9900A0BE0FD12746D8042900A0BE060108A
:20474000900858E0FBA3E0FAA3E0F9127AD9801C90086D7401F0A3740AF0A3740CF090086E
:2047600058E0FBA3E0FAA3E0F9126B6C800E900858E0FBA3E0FAA3E0F9127B8A900869EFCB
:20478000F0803190086D7401F0A3740AF0A37410F0900858E0FBA3E0FAA3E0F91270F5901B
:2047A0000869EFF0900A10E090095AF0900A11E090095BF0129BE19009577446F0A3740589
:2047C000F0900869E0900959F0900A5EE0FBA3E0FAA3E02401F9E43AFA129E3C900A5DF04A
:2047E000A37401F0A37409F0A37457F00298BC7F05129744900AD2129740900AD3EFF022B9
:2048000090087E7480F0E4900880F0A3F0900824E0FCA3E0FD24F0FBEC34FFFAD3EB94E8A5
:20482000EA9403401BED2410FFE43CFEEF7806CEC313CE13D8F9FF7C007D30129E898016A4
:204840007C007D30AF03AE02129E89EF7806CEC313CE13D8F9FF90084BEEF0A3EFF0125F1E
:2048600061E4FF128645129BA9AA06AB07900846E0FEA3E0FFD394E8EE9403401BEF2420BF
:20488000FFE43EFEEF7806CEC313CE13D8F9FF7C007D30129E89801A900846E0FEA3E0FFFD
:2048A0007C007D30129E89EF7806CEC313CE13D8F9FFD3EF9BEE9A4045129BA9D3EF94E8D6
:2048C000EE9403401A129BA9EF2418FFE43EFE7C007D30129E9B7C007D41129E89800F12D1
:2048E0009BA97C007D41129E897D30129E9BC3900847E09FFF900846E09EFE1287DF900087
:204900000FE0700C90085CE07003127A277F0A22900849A3E090087DF0E490087CF09000A6
:204920000FE0FF900849E475F001129F26FCC3E5F09FEC94004007E4900849F0A3F09008AD
:2049400049E0FEA3E07802C333CE33CED8F92410F58274003EF583E0FCA3E0FDA3E0FEA348
:20496000E0FF90088312A1067F16121D9F900849E0FEA3E024E4F58274003EF583E0D3641F
:20498000809458404F900855E0FEA3E0FF9008877401F0A37408F0A3747EF07B017A087940
:2049A0007F125800900849E0FEA3E024E4F58274003EF583E0FF90087EE0FED3EF6480F8B2
:2049C000EE648098400E90087CE004F0E0C394355002211E900849E0FEA3E024E4F5827405
:2049E000003EF583E0FF90087EE0FED3EF6480F8EE6480985010129A0AE490084EF07F01D6
:204A00001286457F002290084E7401F0E4FF12864590085CE07003127A277F0A22D292D232
:204A2000937B017A0879757D089008A3EBF0A3EAF0A3E9F0A3EDF0E4A3F09008A6E075F0E9
:204A400008A4FF9008A8E5F0F0A3EFF0A3E4F0A37410F0E4A3F0A37480F078AE7C087D0170
:204A60007BFF7AB1798A7E007F02129DF49008A3E0FBA3E0FAA3E0F9E4129E777FE87E03EA
:204A800061139008A8E07002A3E070026118209505E59130E7F8E59120E77D3081229008FE
:204AA000A3E0FBA3E0FAA3E0F99008ACE0FFE92FF9E43AFA129E3CFF9008ADE04F129E77AD
:204AC0007F1E7E001297DB9008A9E024FFF09008A8E034FFF09008ADE0FFC313F0702374CF
:204AE00080F09008ACE004F09008A3E0FBA3E0FAA3E0F99008ACE0FFE92FF9E43AFAE412DD
:204B00009E77309505E59130E7F8E59120E7097F1E7E001297DB4182E49008ACF0A374809A
:204B2000F09008AAE4F0A37410F09008A8E07002A3E0600261BA9008AAE07002A3E0607AD5
:204B4000209505E59130E7F8E59120E76D30811F9008ACE024AEF582E43408F583C083C054
:204B600082E0FF9008ADE0FEEF4ED082D083F07F1E7E001297DB9008ABE024FFF09008AAC8
:204B8000E034FFF09008ADE0C313F070157480F09008ACE004F0E024AEF582E43408F583E5
:204BA000E4F07F1E7E001297DB309505E59130E7F87F1E7E001297DB61361294C49008A853
:204BC000E0FCA3E0FD4C7008A3E07002A3E060179008A6E075F008A4B5050AECB5F006A399
:204BE00074FDF0802D80259008A3E0FBA3E0FAA3E0F9A3E0FD7C001281C3EFF4FFEEF4FEDF
:204C00009008AEE06E7003A3E06F60069008A774FFF09008A7E0FF22900A5D7440F0A374A1
:204C200001F0A37409F0A37457F09009577444F0A37440F0EF6401705D7F0112955712483D
:204C400000E4900002F0900822F0A3F0EF703F7B0190086D04F0A37408F0A37426F0E4A3DB
:204C6000F0900857E0900871F0A374FFF0A37499F0A374BBF0900119E0900875F07A017999
:204C80001A7D2D12552E900822EEF0A3EFF0E4900119F0129BE1900002E0FFD3900823E0B6
:204CA0009F900822E094005002A1BE900002E0FD75F028A4243EF582E5F03401F583E0FE9D
:204CC000240A900958F0EE240290095EF075F028EDA4241CF582E5F03401F583E090095F9B
:204CE000F0900002E075F028A4241DF582E5F03401F583E0900960F0EF75F028A4241EF9C3
:204D0000740135F0FA7B01C0039008CAEBF0A37409F0A37461F0900002E075F028A4243E06
:204D2000F582E5F03401F583E09008CDF0D003123FBF900002E075F028A42441F582E5F00E
:204D40003401F583E090095AF0900849E0FEA3E07802C333CE33CED8F9FBAA062410F5823B
:204D600074003AF583A3A3A3E0FF90095BEFF074102BF58274003AF583E0FCA3E0FDA3E047
:204D8000FEA3E0FF780812A0E090095CEFF0900849E0FEA3E07802C333CE33CED8F9241027
:204DA000F58274003EF583E0FCA3E0FDA3E0FEA3E0FF781012A0E090095DEFF0800B9009E0
:204DC000587405F0E490095BF0900822E0FEA3E0FF4E600A900002E0FEC3EF9E8001E490C3
:204DE0000959F0900002E004F022FDF0900894E0FF3395E0FEEF25E0FFEE33FE746D2FF920
:204E0000740A3EFA7B019008A8EBF0A3EAF0A3E9F09008A8E0FBA3E0FAA3E0F9E4129E772D
:204E20009008A8E0FBA3E0FAA3E02402F9E43AFAE4129E779008A8E0FBA3E0FAA3E02401D5
:204E4000F9E43AFA7408129E779008A8E0FBA3E0FAA3E02403F9E43AFA7408129E77ED902B
:204E600008A830E70FE0FBA3E0FAA3E0F9129E3C4480800DE0FBA3E0FAA3E0F9129E3C4447
:204E800040129E77ED9008A830E60FE0FBA3E0FAA3E0F9129E3C4420800DE0FBA3E0FAA3AD
:204EA000E0F9129E3C4410129E77ED9008A830E50FE0FBA3E0FAA3E0F9129E3C4408800DC8
:204EC000E0FBA3E0FAA3E0F9129E3C4404129E77ED9008A830E40FE0FBA3E0FAA3E0F9126D
:204EE0009E3C4402800DE0FBA3E0FAA3E0F9129E3C4401129E77ED9008A830E314E0FBA307
:204F0000E0FAA3E02402F9E43AFA129E3C44808012E0FBA3E0FAA3E02402F9E43AFA129EF9
:204F20003C4440129E77ED9008A830E214E0FBA3E0FAA3E02402F9E43AFA129E3C44208055
:204F400012E0FBA3E0FAA3E02402F9E43AFA129E3C4410129E77ED9008A830E114E0FBA3F6
:204F6000E0FAA3E02402F9E43AFA129E3C44088012E0FBA3E0FAA3E02402F9E43AFA129E11
:204F80003C4404129E77ED9008A830E014E0FBA3E0FAA3E02402F9E43AFA129E3C44028051
:204FA00012E0FBA3E0FAA3E02402F9E43AFA129E3C4401129E777F0222900A0AE0600CA33F
:204FC000E090085CF09001197401F0900957745EF0A37403F0900A5E7401F0A37409F0A332
:204FE0007457F0900A5D7440F090085CE0900959F01298BC90085CE07003127A27222222DF
:20500000900894EBF0A3EAF0A3E9F0A3EDF0A37412F07F8F129A757F96129A7575088F7511
:205020000990900897E0FD2403FFE433FEEF7804CEA2E713CE13D8F87830F6ED2403540FF5
:20504000C454F0440B08F6900897E033333354F8FFF0900B08E025E0540E44A008F60876CE
:2050600012900897E0FEC4540F08F6EEC454F008F67E05EFC39408403A74302EF8C000E63D
:20508000FD900894E0FBA3E0FAA3E0F9129E3CFCC4540F4DD000F60EECC454F0FD74302E20
:2050A000F8A60574F82FFF900895E475F001129F2680C074302EF8E6F6900897E0FF13134B
:2050C00013541FF0E02406F0900899E4F0A37400F0A37430F0900897E0D3941A5002219189
:2050E000530EBF9008A0741DF0900899E0F9A3E0FAA3E09008A1C9F0A3EAF0A3E9F0A374CB
:205100001AF07B007A0079097D01128F92900897E024E6F090089AE475F01A804A900898C5
:20512000E0FF900897E0D39F40427D0F7C007F007E401291BA530EBF900899E0FBA3E0FA42
:20514000A3E0F9900898E09008B7F07F1F128DAE900897E0FFA3E0FEC3EF9E900897F0EEAD
:20516000FF90089AE48FF0129F2680B17D0F7C007F007E401291BA900899E0FBA3E0FAA3C5
:20518000E0F9900897E09008B7F07F1F128DAE802E9008A0741DF0900899E0F9A3E0FAA36C
:2051A000E09008A1C9F0A3EAF0A3E9F0900897E09008A4F07B007A0079097D01128F927D44
:2051C0000F7C007F807E001291BA7F96029A75E4900869F0900A0AE0640170677F02129587
:2051E0005712480090086AEFF0E4900000F0128E0690086AE06009E4900822F0A3F08032F5
:20520000900A0BE090086FF0A37401F0A3740AF0A3740CF0900A14E0900873F07B017A0166
:20522000791A7D2D124268EF3395E0900822F0A3EFF0129BE19008587401F0A37401F0A324
:20524000741AF0E4900869F0900869E0FFC3940F501474572FF582E43409F583E4F09008DB
:2052600069E004F080E29009577440F0A37410F0E490095AF0900000E0FB75F028A4243E1F
:20528000F582E5F03401F583E0FA90095BF0900849E0FEA3E07802C333CE33CED8F92410D1
:2052A000F58274003EF583E0FCA3E0FDA3A3E0FF900964EFF0900849E0FEA3E07802C3333E
:2052C000CE33CED8F92410F58274003EF583E0FCA3E0FDA3E0FEA3E0FF780812A0E090094F
:2052E00065EFF0900849E0FEA3E07802C333CE33CED8F92410F58274003EF583E0FCA3E0E4
:20530000FDA3E0FEA3E0FF781012A0E0E4900966EFF0EA603AEB75F028A4241EF97401352C
:20532000F0FA7B01C0039008CAEBF0A37409F0A3745CF0900000E075F028A4243EF582E535
:20534000F03401F583E09008CDF0D003123FBF900822E0FEA3E0FF4E600E900000E0FEC391
:20536000EF9E900959F080099009587405F0E4A3F0900000E004F0900A5D7410F0A374017D
:20538000F0A37409F0A37457F00298BC90086AEBF0A3EAF0A3E9F0A3EDF0900875740DF085
:2053A000E4900874F0FD7F1A1299167D187F1B129916900871E0FF14F0EF7002A11F900821
:2053C00074E06002A11F128A04C292D293D2937F017E001287DF127971900872EFF0339576
:2053E000E0FEEF25E0FFEE33FE746D2FF9740A3EFA7B01900875E0FD124E06900872E02F19
:20540000F0900875E0A3F0E4900873F090086AE0FBA3E0FAA3E0F9900873E0FFFD3395E0D8
:20542000FCE92DF9EA3CFA129E3CFEEF3395E0FC74772DF58274083CF583EEF0900872E03D
:20544000FF3395E0FEEF25E0FFEE33FE746D2FF9740A3EFA7B0174772DF58274083CF5839B
:20546000E0FD124E06900872E02FF0A3E004F0E0C364809488409590086DE0FD90087FF008
:20548000900872124DEF900872E02FF090086DE004F0A3E0FBA3E0FAA3E0F9129E3CFD90E2
:2054A0000880F0900872124DEF900872E02FF090086FE475F001129F267B017A0879767D81
:2054C0000B7C001281C390087212905C900872E02FF07B017A0A796DE0FD3395E0FC1298CD
:2054E000E7D293D292D2937B017A0879817D01124A29900874EFF0700E900881E07FFC704F
:2055000001FF900874EFF0128A04C292D293D2937F0F7E001287DF1296141294C461B29095
:205520000874E06003129C2D900874E0FF22900869EBF0A3EAF0A3E9F0A3EDF0E49008767D
:20554000F0A3F090087AF0F50EF50F7F8F129A75E490087AF090086CE0FF90087AE0C39F73
:20556000504D900869E0FBA3E0FAA3E0F990087AE0FF75F028A4F582E92582F9EA35F0FA8E
:20558000E4F5F0129F7DEF75F028A4FF900869E0FBA3E0FAA3E02FF9EA35F0FAE92424F9BE
:2055A000E43AFAE4129E7790087AE004F080A6E4F50EF50F900875E0601190086DE0FBA3F0
:2055C000E0FAA3E0F9A3E0FD1250007F2C7E01129C66E4F50EF50F900871E0FF12898790D0
:2055E000087B7401F0A37499F0E47F01FEFDFC900871E0F9F812A0F3900878EEF0A3EFF0D9
:2056000090086CE0FD900876E0FEA3E0FFC39DEE9400505E900879E024FFF0900878E03483
:20562000FFF07C007D28129E89900869E0FBA3E0FAA3E02FF9EA3EFA90087CE0FD122CB01C
:20564000BF010E900877E004F07006900876E004F0900872A3E0FAA3E0F912A15890087B20
:20566000EFF0900878E07002A3E0600690087BE0708E7F807E001298317F96129A757F8F73
:20568000129A75E4F50EF50F900876E07002A3E07021900B0DE024FFF0900B0CE034FFF045
:2056A000E07002A3E07015FF128645129C2D1244AE8000900B0CE4F0A3740AF0900876E0DB
:2056C000FEA3E0FF2290086AEBF0A3EAF0A3E9F0E4900872F090086AE0FBA3E0FAA3E02473
:2056E00025F9E43AFA9008907401F0A37408F0A37473F01275EA900871EFF06003E0FF22A1
:2057000075088F900872E0FF7003750990EFB40103750991E47830F60876570876C490082C
:205720006DE0FBA3E0FAA3E0F9129E3CFF900873E06F08F6E92401F9E43AFA129E3CFF904B
:205740000874E06F08F690086AE0FBA3E0FAA3E02425F9E43AFA129E3CFF131313541FFEB4
:20576000900870E0C43354E04E08F690086AE0FBA3E0FAA3E02426F9E43AFA129E3CFE1395
:205780001313541FFDEFC43354E04D08F6EEC43354E008F67D367F0D1299167F8F129A75C8
:2057A000E4F50EF50F9008A0741DF0A3E4F0A37400F0A37430F0A37408F07B007A0079090A
:2057C0007D01128F9290086A1282EC900871EFF07D3F7F0D129916900871E0FF60012290AA
:2057E000086EE475F002129F26900872E004F0E0C394025002C1D57F0022E4900B43F0229D
:20580000900884EBF0A3EAF0A3E9F0EEC313FEEF13FF90088EEEF0A3EFF04E700790088E64
:20582000F0A304F0E4FF12974490088AEFF07D02E4FF1299167F0912974490088DEFF07DF7
:20584000FF7F0912991690088AE020E1077F0A7E001287DFE4900890F090088E74FFF5F0FD
:20586000129F3C45F060481299E490088BEFF0E0FFC4540FFEEF540F2EFF900891F0900899
:2058800090E0FD3395E0FCD3EF9DEC6480F874809840C6A3E0900890F090088BE0FF900809
:2058A00084E0FBA3E0FAA3E0F9EF129E7780AA900890E0FF701E900887E0FBA3E0FAA3E0C1
:2058C000F97480129E77900884E0FBA3E0FAA3E0F9E4216DEF7803A2E713D8FBFF90089052
:2058E000E02FF07F0A12974490088CEFF07F0512974490088CE0FE30E211900890E024B5B9
:20590000F0EE30E023E02405F0801D900890E024B9F0EE30E104E024F6F090088CE030E00A
:2059200007900890E02408F0EF30E71C900890E0FF90088CE0C41313540375F003A4FEC301
:20594000EF9E900890F0801490088CE0C41313540375F003A4FF900890E02FF0900890E08F
:20596000FF900887E0FBA3E0FAA3E0F9EF129E7790088DE0FD7F0912991690088A129912F5
:2059800090088AE030E0077F067E001287DF22900B38E024DF7002417314700241912421D8
:2059A000B40500400241AB9059B125E0500205837321BB21CE21F34122413C900B3374FF14
:2059C000F0A374A9F0A37416F090A9168065900B3374FFF0A374A9F0A37428F090A92BE47E
:2059E00093FE90A92AE4937C002400FFEC3E900B40418B900B39E075F003A42467F582E525
:205A0000F0340BF583E0FBA3E0FAA3E0F9900B33EBF0A3EAF0A3E9F0129E3CFF900B40E4BF
:205A20008069900B3374FFF0A374A9F0A37431F090A931E493FF900B40E4804F900B39E042
:205A4000FF64817066EF900B33B4811074FFF0A374A9F0A37443F090A943800E74FFF0A31D
:205A600074A9F0A3744AF090A94AE493FF900B40E48018900B3374FFF0A374A9F0A3743A46
:205A8000F090A93AE493FF900B40E4F0A3EFF0801D900B3374FFF0A374A9F0A37451F09096
:205AA0000B407403F0A37414F080031217E3900B38E0FF64016013EF6402600EEF64036087
:205AC00009EF64046004EFB40523900B3DE0FFD3900B41E09F900B40E094004010900B3CDC
:205AE000E0700AE0FE900B40EEF0A3EFF0900B42E064046018E59620E7FB759611759740B1
:205B0000900B427401F0E4900B3EF0A3F02290086DEFF0A3ECF0A3EDF0A3EAF0A3EBF0E41F
:205B200090087BF0FE7F2CFDFB7A00793012A335783276D490086DE033333354F808F6FDFB
:205B4000A3E0FAA3E0FBEAFFEF540325E0FFED4FFFF6FDEBAE027807CEA2E713CE13D8F8B4
:205B600054014D7833F690086EA3E0FF25E054FE08F6A3E064827004A3E0646660028105F3
:205B8000900870E0FCA3E0FDECC41313135401783446F6EDAE047807CEC313CE13D8F9788F
:205BA00035F6900871E025E0FFE43308A607787C7C087D017BFF7AA779857E007F02129DC4
:205BC000F4900883E4F0A37410F0A3E4F0A37400F0A37436F0A3E4F0A37407F07B017A088D
:205BE000797CE4FDFC1210479008837401F0A37456F0A3E4F0A37400F0A37438F0A3E4F059
:205C0000A374078054900870E0FCA3E0FDEC131313541F783446F6EDAE047803CEC313CE22
:205C200013D8F97835F6900870E0FEA3E07805C333CE33CED8F97836F6900870E0FFA3E053
:205C4000900883CFF0A3EFF0A3E4F0A37400F0A37436F0A3E4F0A37403F0900872E0FBA324
:205C6000E0FAA3E0F9E4FDFC121047900875E0F9A3E0FAA3E0900875C9F0A3EAF0A3E9F0E3
:205C8000A3E4F0A3F0A3F0A3E0FF227A087975E4FD90088CEBF0A3EAF0A3E9F0A3EDF0906A
:205CA00008A27451F0900893E02402F0E0FFD394204007EFC41354078001E4FD7F1A1299F0
:205CC00016900893E0541F75F008A4FD7F1B129916900893E024FEF0128A04C292D293D27F
:205CE000937F017E001287DF127971900894EFF03395E0FEEF25E0FFEE33FE746D2FF9745F
:205D00000A3EFA7B019008A2E0FD124E06900894E02FF09008A2E0900897F0E4900895F0E3
:205D200090088CE0FBA3E0FAA3E0F9900895E0FFFD3395E0FCE92DF9EA3CFA129E3CFEEFB6
:205D40003395E0FC74982DF58274083CF583EEF0900894E0FF3395E0FEEF25E0FFEE33FE1E
:205D6000746D2FF9740A3EFA7B0174982DF58274083CF583E0FD124E06900894E02FF0A3F7
:205D8000E004F0E0C364809488409590088FE09008A0124DEA900894E02FF0900893E014E5
:205DA0009008A1124DEA900894E02FF07B017A0879977D0B7C001281C390089412905C9014
:205DC0000894E02FF07B017A0A796DE0FD3395E0FC1298E7D293D292D293900890E0FBA35C
:205DE000E0FAA3E0F9A3E0FD124A29900896EFF06003129C2D900896E0FF2290087FEBF0DC
:205E0000A3EAF0A3E9F0E4900885F090087FE0FBA3E0FAA3E02425F9E43AFA9008907401AF
:205E2000F0A37408F0A37486F01275EAEF6006E4F50EF50F2275088F750990E47830F6085F
:205E400076500876C6900882E0FBA3E0FAA3E0F9129E3CFF900886E06F08F6E92401F9E409
:205E60003AFA129E3CFF900887E06F08F690087FE0FBA3E0FAA3E02425F9E43AFA129E3C5F
:205E800008F690087FE0FBA3E0FAA3E02426F9E43AFA129E3C08F67F8F129A75E4F50EF5C2
:205EA0000F9008A0741DF0A3E4F0A37400F0A37430F0A37407F07B007A0079097D01128FC1
:205EC00092E4F50EF50F7F5FFE129831E50F20E0727F1C129744EF540FFFC3940340027F34
:205EE000037B017A087988128C6290087FE0FBA3E0FAA3E02426F9E43AFA129E3CFF9008D0
:205F000089E06F703690087FA3E0FAA3E02425F9E43AFA129E3CFF900888E0B5071D7F8FC0
:205F2000129A75E4F50EF50F90088375F002129F26900885E0B401137F0022E4F50EF50FAB
:205F40007F02229008857402F0FF22E4F50EF50F900885E004F0E0C394025002C10B7F0048
:205F600022E49008A7F030A102E1FED2A17F0C7E001287DFE49008A7F0900AD6E054FCFD96
:205F8000E4FF1299169008A67401F09008A6E0FFC394195059EF64126013EF6414600EEFE8
:205FA00064156009EF64166004EFB417269008A7E0FF04F0EF75F003A424F3F9740A35F092
:205FC000FA7B019008A6E0FF9008B77403F0128DAE80139008A6E0FF24D6F582E4340AF5F3
:205FE00083E0FD1299169008A6E004F0809D7F2C7E01129C66127000900AD6129912222220
:2060000090087FEDF090087CEBF0A3EAF0A3E9F0900887E4F0A37421F0E92425F9E43AFA46
:206020009008907401F0A37408F0A37485F01275EAEF6006E4F50EF50F2275088F7509914A
:20604000E47830F60876650876C390087FE0C4333354C0FF08F6A3E0FE1313543F4FF6EEFB
:20606000C4333354C0FF08F6A3E0FBA3E0FAA3E0F9129E3CFE900885E06EFE1313543F4F13
:20608000F6EEC4333354C0FF08F6E92401F9E43AFA129E3CFE900886E06EFE1313543F4F66
:2060A000F6AF06EFC4333354C0FF08F690087CE0FBA3E0FAA3E02425F9E43AFA129E3CFED8
:2060C0001313543F4FF6EEC4333354C0FF08F690087CE0FBA3E0FAA3E02426F9E43AFA123D
:2060E0009E3CFE1313543F4FF6EEC4333354C008F6900887A3E0FD7F1B129916900887E0A7
:206100005403FD7F1A1299167D3E7F0D1299167F8F129A75E4F50EF50F9008A0741DF0A353
:20612000E4F0A37400F0A37430F0A37409F07B007A0079097D01128F9290087CE0FBA3E0A3
:20614000FAA3E02425F9E43AFA126D7D900884EFF07D3F7F0D129916900884E0FF22900BB0
:2061600083EBF0A3EAF0A3E9F0A3EDF0E4900B88F07BFF7AA77912900B87E09008CAF012C5
:206180003000900B83E0FBA3E0FAA3E02401F9E43AFA129E3C9008CAF0900B83A3E0FAA324
:2061A000E0F9129E3C9008CBF07BFF7AA7791D1230007BFF7AA7792E900B86E02402900853
:2061C000CAF0123000900B83E0FBA3E0FAA3E02403F9E43AFA129E3C9008CAF0900B83A393
:2061E000E0FAA3E02402F9E43AFA129E3C9008CBF07BFF7AA779481230007BFF7AA77956C4
:20620000123000900B86E0FF900B88E0FEC39F5030900B83E0FBA3E0FAA3E02404F9E43A21
:20622000FAEE7E0029F9EE3AFA129E3C9008CAF07BFF7AA7790A123000900B88E004F0809F
:20624000C27BFF7AA77910123000900B83E0FBA3E0FAA3E02424F9E43AFA129E3C9008CA76
:20626000F07BFF7AA7795C123000900B83E0FBA3E0FAA3E02425F9E43AFA129E3C9008CADB
:20628000F0900B83A3E0FAA3E02426F9E43AFA129E3C9008CBF07BFF7AA77972023000900E
:2062A0000A0AE0640170547F01129557124800E4900001F0900822F0A3F0EF703B7B0190A1
:2062C000088204F0A37408F0A37426F0E4A3F0900857E0900886F0A374FFF0A37499F0A367
:2062E00074BBF0A37401F07A01791A7D2D123431900822EEF0A3EFF0129BE1900A5E740133
:20630000F0A37409F0A37457F0900A5D7440F09009577432F0900822E0FEA3E0FF4E600A2C
:20632000900001E0FEC3EF9E8001E4900959F0900001E0FFD3900823E09F900822E09400AC
:20634000500261CD900001E0FD75F028A4243EF582E5F03401F583E0FE2406900958F0EEEC
:20636000240290095AF075F028EDA4241CF582E5F03401F583E090095BF0900001E075F023
:2063800028A4241DF582E5F03401F583E090095CF0EF75F028A4241EF9740135F0FA7B01C7
:2063A000C0039008CAEBF0A37409F0A3745DF0900001E075F028A4243EF582E5F03401F5EF
:2063C00083E09008CDF0D003123FBF800B9009587404F0E490095AF0900001E004F022E40C
:2063E000900869F0A3F0900878F0A3F0A3F0A3F0124800900869EFF0600281D21269269040
:206400000822E07002A3E070089008697409F081D27B017A0A790A128B7B900869EFF06069
:206420000281D2900A0EE0FDC4540FFF90086BE4F0A3EFF0E0F8E4F0E890086BF0ED540F2C
:2064400075F010A4FFE045F0F0A3E04FF0900A0FE0FFC4540FFD90086BE0F0A3E04DF0EF2F
:20646000540F7F00FEA3F0A3EFF0900A10E0FDEDFF90086DEEF0A3EFF0A37401F0A3740A26
:20648000F0A37413F0A37401F0A37409F0A3745BF0900A11E0900875F0900A12E090087656
:2064A000F0E4A3F0FE7F3CFD7B017A09795B12A33590087F7401F0A37408F0A3746BF09075
:2064C0000858E0FBA3E0FAA3E0F9122800900869EFF0129BE19009577460F0A37440F09055
:2064E0000869E0900959F0900877E090095AF07B017A097957900A5EEBF0A3EAF0A3E9F0FC
:206500002401F9E43AFA129E3C900A5DF00298BCE490086AF0900A0CE0900869F012480075
:2065200090086AEFF06002C107126926900822E07002A3E0700890086A7409F0C1079008D9
:2065400069E06002A1D57B0190086B04F0A37409F0A3745BF0900A0BE090086EF090086AB8
:20656000E0705E900869E0C3941E50551299BBEF604F900A0AE0FD90086EE0FF04F090087C
:2065800073EFF0A37401F090086BE0F9A3E0FAA3E0900875C9F0A3EAF0A3E9F0900858E036
:2065A000FBA3E0FAA3E0F9123D4790086AEFF0900869E004F090086CE475F002129F2680F5
:2065C0009C900869E014F090084EE0603A90086A740AF08032900A0AE0FDA3E0900873F0B9
:2065E000900869E0900874F0A37401F0A37409F0A3745BF0900858E0FBA3E0FAA3E0F9126E
:206600003D4790086AEFF0129BE19009577438F090086AE0900959F0900869E0FD25E02430
:2066200004900958F090095AEDF0900A5D7440F0A37401F0A37409F0A37457F00298BC122C
:20664000480090086CEFF06002E12D126926900822E07002A3E0700890086C7409F0E12D78
:20666000128B7590086CEFF06002E12D900A0AE0FFB401057402F0800AEFB40206900A0A39
:206680007401F0E4900869F0A3F0A3F0900A0BE0FD701090086974C0F0900A0AE0FEC454D9
:2066A00030802BEDB401139008697430F0900A0AE0FF25E025E0540C8014900A0BE0FDB4FE
:2066C0000212900869740CF0900A0AE0540390086AF08038EDB403129008697403F0900AF8
:2066E0000AE0FFC4333354C08015900A0BE0B4041490086A74C0F0900A0AE0FFC45430900C
:20670000086BF08007E4900869F0A3F09008707401F0A37408F0A37469F0900858E0FBA3CD
:20672000E0FAA3E0F91272C990086CEFF0129BE1900957743CF0A37404F090086CE090092D
:2067400059F0900A5EE0FBA3E0FAA3E02401F9E43AFA129E3C900A5DF0A37401F0A37409EC
:20676000F0A37457F00298BC900869EFF0D3940F40037489F0900869E02457F582E4340BF9
:20678000F583E090086BF0E0C413540790086AF090086AE0FFD39400404DC2A2EF14FF74FB
:2067A000017E00A807088005C333CE33CED8F9FF90086BE0FDEF5D7BFF600D7AA6797A1251
:2067C00030007FC27E01800B7AA6797C1230007FFA7E001287DFD2A27F5E7E011287DF90A0
:2067E000086AE014F080A97BFF7AA6797E900869E09008CAF01230007FC27E010287DF22CA
:20680000E4900869F0128E06124800900869EFF0E4900822F0A3F0EF600201D190086B0478
:20682000F0900882F0A3740AF0A3740BF0900A0AE0900885F0E4A3F0A374FFF0A37499F08D
:20684000A374BBF0A37401F0FB7A01791AFD123431900822EEF0A3EFF0E490086AF0900A67
:206860000AE0FF90086AE0FEC39F501A740B2EF582E4340AF583E06005E490086BF0900811
:206880006AE004F080D8900822E07002A3E0704190086BE0603B9008827401F0A3740AF014
:2068A000A3740BF0A3EFF0900857E0900886F0A374FFF0A37499F0A374BBF0E4A3F07B010C
:2068C0007A01791A7D01123431900822EEF0A3EFF0129BE1900822E07002A3E0900858602E
:2068E000127401F0A37401F0A3741AF0E4900869F0800CE4F0A3F0A3F09008697409F0909F
:2069000009577434F0A37403F0900869E0900959F0900A5D7403F0A37401F0A37409F0A399
:206920007457F00298BC900858A3E0FAA3E04A7003FEFF22900858E0FBA3E0FAA3E0240487
:20694000F9E43AFA900882EBF0A3EAF0A3E9F0900858A3E0FAA3E02424F9E43AFA129E3C03
:20696000900885F0E4A3F0A374FFF0A37499F0A374BBF0A37401F0FB7A017942FD1234317E
:20698000900822EEF0A3EFF090087D7401F0E490087CF0900858E0FBA3E0FAA3E02424F96F
:2069A000E43AFA129E3CFF90087CE0FEC39F5028900858A3E0FAA3E02404F9E43AFAEE7C75
:2069C0000029F9EC3AFA129E3C6005E490087DF090087CE004F080BB900822E07002A3E089
:2069E000704E90087DE06048900858E0FBA3E0FAA3E02404F9E43AFA900882EBF0A3EAF0C6
:206A0000A3E9F0A3EFF0900857E0900886F0A374FFF0A37499F0A374BBF0E4A3F07B017AC6
:206A20000179427D01123431900822EEF0A3EFF0900822E07002A3E0600E9008587401F039
:206A4000A37401F0A37442F02290084DE024FD604B147002611E24026002615AE490000A6C
:206A6000F0FFFEFDFC90000612A106900A097402F0121027EF70026160129CBF90000AE086
:206A8000FE04F074082EF582E4340AF583EFF090084D7403F0E490085CF06160900006E01F
:206AA000FCA3E0FDA3E0FEA3E0FFE4FAF9F8EF2401FFEA3EFEE93DFDE83CFC90000612A1C3
:206AC00006E4FF7E80FDFC900006E0F8A3E0F9A3E0FAA3E0FBD312A0B9501390000AE0FFD7
:206AE000943F500A900A09E0FEEFC39E400790084D7404F022121027EF6065129CBF9000E8
:206B00000AE0FE04F074082EF582E4340AF583EFF0E4FFFEFDFC90000612A10680427F4055
:206B2000900957E4F0A3DFFC7F4090084D7402F090084814F0125F61900A08E075F003A4C5
:206B40002486F582E5F034ACF583740193FA740293F912A158E4900848F090084D7402F0D9
:206B600090085CE060057F01129BCF2290086AEBF0A3EAF0A3E9F02425F9E43AFA90089066
:206B80007401F0A37408F0A37471F01275EAEF6006E4F50EF50F2275088F750991E478308F
:206BA000F60876800876E008760290086DE0FBA3E0FAA3E0F9129E3CFF900871E0FE6F08E1
:206BC000F6E92401F9E43AFA129E3CFF900872E0FD6F08F690086DE0FBA3E0FAA3E024025B
:206BE000F9E43AFA129E3CFFEE6F08F690086DE0FBA3E0FAA3E02403F9E43AFA129E3CFF3B
:206C0000ED6F08F690086AE0FBA3E0FAA3E02425F9E43AFA129E3C08F690086AE0FBA3E099
:206C2000FAA3E02426F9E43AFA129E3C08F67D367F0D1299167F8F129A75E4F50EF50F90E8
:206C400008A0741DF0A3E4F0A37400F0A37430F0A3740AF07B007A0079097D01128F92908D
:206C6000086A1282EC900870EFF07D3F7F0D129916900870E0FF2290087CEFF07F05129709
:206C80004490087E12974090087DEFF0543CF030E21A90087CE02448F0E0D36480948540D1
:206CA00037E024FBF0A3E04401F0802C90087CE02442F0E0C3648094884009E024F8F0A385
:206CC000E04401F090087CE0D3648094765009E0240AF0A3E04402F090087CE0FDD3648032
:206CE0009480403190087EE0547FF0ED75F003129E1A90087FF0D3940340037403F0900884
:206D00007CE0FF90087FE075F003A4FEC3EF9E90087CF0803B90087EE04480F090087CE06A
:206D2000FF3395E0FEC374029FFFE49EFE7C007D03129EF090087FEFF0D3940340037403A1
:206D4000F090087FE075F003A4FF90087CE02FF090087DE0FF90087FE0C4333354C0FEEF18
:206D60004E90087DF0A3E0FD7F0512991690087DE0FD7F0A12991690087CE0FF2290088989
:206D8000EBF0A3EAF0A3E9F0A37404F0900890E4F0A37429F07F807E00129831E4F50EF5B4
:206DA0000F7F8F129A757D147C007F5A7E001291BAE50F30E355900890A3E0FD7F1B12998B
:206DC00016900890E05403FD7F1A1299167F527E001298317F1C129744EF540F900892F0C9
:206DE000C3940340037403F0900892E0FF7B017A08798D128C627F8F129A757D3F7F0D12F9
:206E0000991690088DE04480FFF022E50F30E6567F1C129744EF540F900892F0C3940240FC
:206E2000037402F0900892E0FF7B017A08798D128C627F8F129A75900889E0FBA3E0FAA391
:206E4000E0F9129E3CFF90088DE06F6012E92401F9E43AFA129E3CFF90088EE0B50717E4C1
:206E600090088CF08010E50F90088C30E405740BF080037404F0E4F50EF50F90088CE0FFF5
:206E80002290088DEBF0A3EAF0A3E9F0AC0712797190089CEFF0E4900891F0EF3395E0FE83
:206EA000EF25E0FFEE33FE746D2FF9740A3EFA7B01E4FD124E0690089CE02FF0900890E003
:206EC000900892F0FD90089C124DEF90089CE02FF0AF04900893EFF0FD90089C124DEF901A
:206EE000089CE02FF0A37403F090089DE0FFC36480948B505B90088DE0FBA3E475F0011261
:206F00009F3CA9F0FA129E3CFEEFFD3395E0FC74912DF58274083CF583EEF090089CE0FFBF
:206F20003395E0FEEF25E0FFEE33FE746D2FF9740A3EFA7B0174912DF58274083CF583E0A5
:206F4000FD124E0690089CE02FF0A3E004F080997B017A0879917D0B7C001281C3AD07AC49
:206F60000690089C12906090089CE02FF07B017A0A796DE0FD3395E0FC0298E79008697445
:206F8000FFF0124800900869EFF07029900A12E0FD9008907401F0A37409F0A3745BF09017
:206FA0000A13E0900893F07B017A0A790A125C91900869EFF0129BE1900957744AF0A37414
:206FC00040F0900869E0FF3395E0FE7CFF7DFF129E89900959EFF0900A13E090095AF07B0F
:206FE000017A097957900A5EEBF0A3EAF0A3E9F02401F9E43AFA129E3C900A5DF00298BC12
:20700000900AF2E0700201F47B017A0879A87D037F121293EE9008AAE054FEF09008A9E055
:20702000543FF04440F07B017A0879A89008B77403F07F12128DAEE49008ACF0A3F0900863
:20704000ADE004F070069008ACE004F07F647E00129C667F0E1297449008ABEFF020E10F00
:20706000C39008ADE094649008ACE0940040CF7A0879A81293E89008A9E04408128D9F7F0F
:20708000C87E00129C667F10129744EF54079008AEF09008A9E054F7128D9F9008AEE0FFCB
:2070A000D394014005EF9406404AE49008ACF0A3F09008ADE004F070069008ACE004F0902E
:2070C00008A9E0547F128D9F9008A9E04480128D9F7F0A7E001287DF7F0E1297449008ABAF
:2070E000EFF020E10FC39008ADE094039008ACE0940040BD2290086AEBF0A3EAF0A3E9F075
:207100002425F9E43AFA9008907401F0A37408F0A37470F01275EAEF6006E4F50EF50F222F
:2071200075088F750991E47830F60876700876E008760708F690086DE0FBA3E0FAA3E0F90A
:20714000129E3CFF900870E06F08F6E92401F9E43AFA129E3CFF900871E06F08F690086A8D
:20716000E0FBA3E0FAA3E02425F9E43AFA129E3C08F690086AE0FBA3E0FAA3E02426F9E4EC
:207180003AFA129E3C08F67D367F0D1299167F8F129A75E4F50EF50F9008A0741DF0A3E477
:2071A000F0A37400F0A37430F0A37409F07B007A0079097D01128F9290086AE0FBA3E0FA0F
:2071C000A3E02425F9E43AFAC002C001A3E0F9A3E0FAA3E0900875C9F0A3EAF0A3E9F0D044
:2071E00001D00212780022900BA3EFF0A37403F0A374E8F0900A5DE0FFA3E0FBA3E0FAA386
:20720000E02401F9E43AFAEF129E77900B43E064017031900B43E0B40117900BA474FFF54D
:20722000F0129F2645F060097F647E00129C6680E2900BA4E07002A3E070097BFF7AA87970
:20724000E8123000E4900BA3F0A2AF9200C2AFE59620E7FB75960E759701E59620E7FB7509
:207260009691E59620E7FBAF97900B43E0FEB4030DE59620E7FB7596117597108046EE70CB
:2072800043900B4304F0EF30E50BE59620E7FB759611759740EF30E20BE59620E7FB759651
:2072A00011E4F597900A5DE0FD7C00A3E0FBA3E0FAA3E0F97F211290B8E59620E7FB759604
:2072C00011759701A20092AF2290086DEBF0A3EAF0A3E9F075088F750991E47830F6087697
:2072E000590876C5A3E0FBA3E0FAA3E0F9129E3C08F6E92401F9E43AFA129E3C08F69008F0
:207300006DE0FBA3E0FAA3E02425F9E43AFA129E3CFFC4540FFE900870E0FBA3E0FAA3E0D8
:207320002402F9E43AFA129E3C54F04E08F690086DE0FBA3E0FAA3E02426F9E43AFA129EAF
:207340003CFEC4540FFDEFC454F04D08F6EEC454F008F67D367F0D1299167F8F129A75E486
:20736000F50EF50F9008A0741DF0A3E4F0A37400F0A37430F0A37408F07B007A0079097D95
:2073800001128F9290086D1282EC900873EFF07D3F7F0D129916900873E0FF22E490086C4D
:2073A000F0900A09E090086BF012480090086CEFF0E07076126926900822E07002A3E070C4
:2073C0000890086C7409F08061128B7590086CEFF0E07056900A10E0900869F0FE900A0B9A
:2073E000E0FF9008717401F0A3740AF0A37411F0A3EEF0900A0AE0900875F0A37401F0A36A
:207400007408F0A3746CF0900858E0FBA3E0FAA3E0F91278B990086AEFF0900869E06F60F5
:207420000990086CE0700374FFF0129BE19009577436F0A37404F090086CE0900959F09010
:20744000086AE090095AF0900A5EE0FBA3E0FAA3E02401F9E43AFA129E3C900A5DF0A37404
:2074600001F0A37409F0A37457F00298BC90086AEBF0A3EAF0A3E9F075088F750991E4780A
:2074800030F60876430876E0087603ED60050876808004E47834F690086AE0FBA3E0FAA3CF
:2074A000E02425F9E43AFA129E3CFF54FEC313783446F6EF5401C43333335480FF90086A21
:2074C000E0FBA3E0FAA3E02426F9E43AFA129E3CFE54FEC3134F08F6EE5401C43333335423
:2074E0008008F67D367F0D1299167F8F129A75E4F50EF50F9008A0741DF0A3E4F0A37400AD
:20750000F0A37430F0A37407F07B007A0079097D01128F9290086A1282EC90086DEFF07D2B
:207520003F7F0D12991690086DE0FF22900B38E07010A3E0700C900B3CE07006A3E0640271
:2075400060031217E3900B36E0247F601314603224027072900B3AE0706CA3E060158066D8
:20756000900B32E0B4040A900B3AE07004A3E060028053900B3374FFF0A374B1F0A3748833
:207580008036900B32E0B40406900B3AE060028035900B3BE0B4812C900B43E0900B33B4A7
:2075A000030C74FFF0A374B1F0A37486800A74FFF0A374B1F0A37488F0900B40E4F0A3740A
:2075C00002F0800580001217E3900B42E064046018E59620E7FB759611759740900B4274D5
:2075E00001F0E4900B3EF0A3F0229008937401F075088F750990E47830F60876300876C11F
:20760000129E3C08F6E92401F9E43AFA129E3C08F6E4F50EF50FFD7F1A1299167D207F1BFE
:207620001299167F8F129A759008A0741DF0A3E4F0A37400F0A37430F0A37405F07B007AEB
:207640000079097D01128F927F807E001298317F8F129A757F5F7E00129831E50F30E62807
:20766000E50F541E60089008937401F08024E4F50EF50F900890E0FBA3E0FAA3E0F9129C73
:20768000EBE4900893F0800AE4F50EF50F90089304F0E4FD7F1B129916E4F50EF50F9008AD
:2076A00093E0FF22900869E4F0A3F0A3F0900AF2E0B4011090086974FFF0A374A8F0A374E0
:2076C00016F08038900A0AE014601304702090086974FFF0A374A8F0A3742AF0801E9008D3
:2076E0006974FFF0A374A8F0A37448F0800E90086974FFF0A374A8F0A3746CF07F31900963
:2077000059E4F0A3DFFC9009577411F0900869E0FBA3E0FAA3E0F91227DBEF04900958F09C
:207720009008CA7401F0A37409F0A37459F0900958E024FE9008CDF0900869E0FBA3E0FA71
:20774000A3E0F9123FBF900A5E7401F0A37409F0A37457F0900A5D7431F00298BCE4FF12FB
:207760009744900883EFF07B017A08797F1293EA90087FE0900882F054CF90087FF07B0108
:207780007A08797F128DA6900883E0440254FEFDE4FF1299167F96129A757F97129A757D0C
:2077A000017F111299167F027E001287DF12996890087EEFF07D027F111299167F027E0029
:2077C0001287DF129968EFFE90087EE0FDEDFF90087CEEF0A3EFF07B017A08797F1293EA59
:2077E000900882E090087FF07B017A08797F128DA690088312991290087CE0FEA3E0FF22DF
:20780000900872EBF0A3EAF0A3E9F09008787404F07F807E00129831E4F50EF50F7F8F12AF
:207820009A757D3F7F0D1299167D147C007F527E001291BAE50F30E675900875E0FBA3E08D
:20784000FAA3E0F97F02128C627B017A0879797F02128C627F8F129A75E50F30E3239008CF
:2078600075E0FBA3E0FAA3E0F9129E3C4480129E77900875E0FBA3E0FAA3E0F9129E3C809B
:2078800029900872E0FBA3E0FAA3E0F9129E3CFF900879E06F6012E92401F9E43AFA129E55
:2078A0003CFF90087AE0B50705E4900878F0E4F50EF50F900878E0FF2290086DEFF0A3EB88
:2078C000F0A3EAF0A3E9F0E4900879F0A3F0900874E0FF90087AE0C39F4002216BE4A3F0C3
:2078E00090087AE0FC90086DE02C900880F0EC75F002A4FF900871E0FBA3E0FAA3E02FF97F
:20790000EA35F0FA900881EBF0A3EAF0A3E9F0900875E0FD90086EE0FBA3E0FAA3E0F9129B
:207920006000900879EFF090087BE004F0E0C39407500C900879E060061299BBEF70A19029
:20794000084EE06006900879740AF0900879E0FF6011900876E0FBA3E0FAA3E0F9EF129E2A
:2079600077800890087AE004F001CE90087AE0FF227B017A0A796D9008A3EBF0A3EAF0A324
:20798000E9F09008A3E0FBA3E0FAA3E0F97455129E779008A3E0FBA3E0FAA3E02402F9E4F6
:2079A0003AFA7455129E779008A3E0FBA3E0FAA3E02404F9E43AFA7473129E779008A3E02B
:2079C000FBA3E0FAA3E02406F9E43AFA740A129E779008A3E0FBA3E0FAA3E02401F9E43A7A
:2079E000FA7408129E779008A3E0FBA3E0FAA3E02403F9E43AFA7408129E779008A3E0FBE3
:207A0000A3E0FAA3E02405F9E43AFA7408129E779008A3E0FBA3E0FAA3E02407F9E43AFA37
:207A20007404129E77FF22E49008A7F020A10241D8E4FF129744900AD6EFF054FCFDE4FF48
:207A40001299169008A67401F09008A6E0FFC394195059EF64126013EF6414600EEF641577
:207A60006009EF64166004EFB417229008A7E0FF04F0EF75F003A424F3F9740A35F0FA7BBF
:207A8000019008A6E0FF7D031293EE80179008A6E0FF1297449008A6E024D6F582E4340A63
:207AA000F583EFF09008A6E004F0809D9008A87401F0A374F4F09008A874FFF5F0129F3C1B
:207AC00045F060127F0E129744EF30E2097F017E001287DF80E0C2A12290086AEBF0A3EAB6
:207AE000F0A3E9F02425F9E43AFA9008907401F0A37408F0A3746EF01275EAEF6006E4F510
:207B00000EF50F2275088F750991E47830F60876400876E008760190086AE0FBA3E0FAA3FC
:207B2000E02425F9E43AFA129E3C08F690086AE0FBA3E0FAA3E02426F9E43AFA129E3C08F5
:207B4000F67D367F0D1299167F8F129A75E4F50EF50F9008A0741DF0A3E4F0A37400F0A33B
:207B60007430F0A37406F07B007A0079097D01128F9290086A1282EC90086DEFF07D3F7F9B
:207B80000D12991690086DE0FF2290086AEBF0A3EAF0A3E9F02425F9E43AFA900890740144
:207BA000F0A37408F0A3746EF01275EAEF6006E4F50EF50F2275088F750991E47830F608D9
:207BC00076400876E008760590086AE0FBA3E0FAA3E02425F9E43AFA129E3C08F690086AEB
:207BE000E0FBA3E0FAA3E02426F9E43AFA129E3C08F67D367F0D1299167F8F129A75E4F55D
:207C00000EF50F9008A0741DF0A3E4F0A37400F0A37430F0A37406F07B007A0079097D01E2
:207C2000128F9290086A1282EC90086DEFF07D3F7F0D12991690086DE0FF22900B8EEBF098
:207C4000A3EAF0A3E9F0900B8EE0FBA3E0FAA3E02402F9E43AFA129E3C9008CAF0900B8E89
:207C6000A3E0FAA3E02403F9E43AFA129E3C9008CBF07BFF7AA679EB1230007BFF7AA6793A
:207C8000FF123000E4900B91F0A3F0900B8EE0FBA3E0FAA3E02424F9E43AFA129E3CFF9038
:207CA0000B91E0FCA3E0FDC39FEC94005034900B8EA3E0FAA3E02404F9E43AFAE92DF9EA0B
:207CC0003CFA129E3C9008CAF07BFF7AA7790A123000900B92E004F070B1900B91E004F0AE
:207CE00080A97BFF7AA7791002300090085BE0B40102E4F0900A0AE06006A3E090084FF063
:207D0000900A0CE06006A3E0900850F0900A0EE06006A3E0900851F0900A10E06006A3E05F
:207D2000900852F0900A12E06006A3E0900853F0900A14E06006A3E0900857F07E007F4086
:207D40007D007B017A09795712A335900957745AF0A37440F090084FE090095AF090085066
:207D6000E090095CF0900851E090095EF0900852E0900960F0900853E0900962F090085736
:207D8000E0900964F0900A5D7440F0A37401F0A37409F0A37457F00298BCC0E0C0F0C0831C
:207DA000C082C0D075D000C000C001C002C003C004C005C006C007E59620E7FB759686E59D
:207DC0009620E7FB9008C3E597F0E59620E7FB759682E59620E7FB9008C4E597F0E596205A
:207DE000E7FB759684E59620E7FB9008C5E597F09008C3E030E103129BF39008C3E030E290
:207E0000031210079008C4E030E0031224CD9008C4E030E1031257FA9008C5E030E10312CE
:207E20007F8B9008C3E030E003129C02D007D006D005D004D003D002D001D000D0D0D082AC
:207E4000D083D0F0D0E032E4900869F0A3F0A3F0A3F0900A0BE090086AF0A3E4F0900A0C0B
:207E6000E0FF90086AE0F0A3E04FF0900A0DE0FAA3E0FFEFFB900A0AE0FF90086AE0FCA39E
:207E8000E0FD9008727401F0A3740AF0A3740FF0A37401F0A37409F0A3745BF0A37401F0ED
:207EA000A37408F0A3746CF0125B0E900869EFF0129BE1900957744EF0A37440F09008696D
:207EC000E0900959F090086CE090095AF07B017A097957900A5EEBF0A3EAF0A3E9F0240159
:207EE000F9E43AFA129E3C900A5DF00298BCE4900B8AF0E4900B8BF0A3F0A3F0900B89F01B
:207F0000900882E4F0A3F0A3F0A3F0900B8AE0900886F0A374FFF0A3749CF0A374FAF0A35A
:207F20007401F0FB7A01791A7D10123431EFFD900B8DE02DF0900B8CE03400F0900B8BE08D
:207F4000FEEFD39E4002EFF0900B89E004F0E0C394FF40AC7BFF7AA6794F900B8AE0900889
:207F6000CAF0900B8CE0FFA3E09008CBCFF0A3EFF0900B8BE09008CDF0123000900B8AE078
:207F800004F0E0C3940F5002C1F322E49008C6F0E59620E7FB75960E759701E59620E7FB2D
:207FA000759694E59620E7FBAF97900B43E0B4030CE59620E7FB75961475972022EF30E6EF
:207FC0000BE59620E7FB75961475978012102F900A48E0FD7C00A37F21128F32900A49E009
:207FE000FBA3E0FAA3E0F9129E3CFF129000E59620E7FB759614E4F59722900A5CE0FF22DB
:20800000E4900B98F0900B98E0FFC3941F400201967BFF7AA4791A9008CAEFF012300090BA
:208020000B98E0FF64126014EF6414600FEF6415600AEF64166005EF6417703C7B017A0B47
:2080400079997D031293EE7BFF7AA47927900B9BE09008CAF01230007BFF7AA47927900B46
:208060009AE09008CAF01230007BFF7AA47927900B99E09008CA8012900B98E0FF129744B3
:208080007BFF7AA4792D9008CAEFF0123000900B98E004F0010522E4FF12974490088212F4
:2080A00093E290087EE0900881F054CF90087EF07B017A08797E128DA6900882E04403FDAB
:2080C000E4FF1299167F96129A757F97129A757D017F111299167F027E001287DF12996836
:2080E000EF3395E090087CF0A3EFF07D027F111299167F027E001287DF129968EFFE900884
:208100007DE0FDEDFF90087CEEF0A31293E2900881E090087EF07B017A08797E128DA69034
:20812000088212991290087CE0FEA3E0FF22900957741DF0900A0AE0FF64126013EF64141E
:20814000600EEF64156009EF64166004EFB417287B017A0879697D031293EE9008CA740167
:20816000F0A37409F0A37459F0A37403F07B017A087969123FBF802E900A0AE0FF12974487
:20818000900869EFF09008CA7401F0A37409F0A37459F0A37401F0FB7A087969123FBFE46D
:2081A00090095AF0A3F0900957741DF0A37406F0900A5DF0A37401F0A37409F0A37457F06E
:2081C0000298BC9008B0EBF0A3EAF0A3E9F0A3ECF0A3EDF074FF9008B7F0A3F0E49008B5B8
:2081E000F0A3F09008B3E0FEA3E0FFC39008B6E09FEE6480F89008B5E06480985051900815
:20820000B0E0FBA3E475F001129F3CA9F0FA129E3CFD9008B7E0FAA3E0FBEAFFEF6D25E08C
:20822000FFE433FE74862FF58274AF3EF583EBFEE4936EFF7401939008B7CFF0A3EFF090BC
:2082400008B6E004F0709C9008B5E004F080949008B7E0FEA3E0FF2290086A7402F0900979
:20826000577458F0E4900869F0900869E0FFC3941F505AEF64126013EF6414600EEF641501
:208280006009EF64166004EFB4171D90086AE07C002457F9EC3409FA7B017D031293EE90BD
:2082A000086AE02403F0801D900869E0FF12974490086AE02457F582E43409F583EFF0900F
:2082C000086AE004F0900869E004F0809C90086AE02402900958F0900A5D7440F0A37401CB
:2082E000F0A37409F0A37457F00298BCE0FBA3E0FAA3E02425F9E43AFA900875EBF0A3EA20
:20830000F0A3E9F0A37404F07F807E00129831E4F50EF50F7F8F129A757D147C007F527E18
:20832000001291BAE50F30E64B7B017A0879797F02128C627F8F129A75E50F30E309900843
:2083400079E04480F08029900875E0FBA3E0FAA3E0F9129E3CFF900879E06F6012E92401BB
:20836000F9E43AFA129E3CFF90087AE0B50705E4900878F0E4F50EF50F900878E0FF2290DE
:208380000BA0EBF0A3EAF0A3E9F07430129E77900BA0E0FBA3E0FAA3E02401F9E43AFA74D3
:2083A00078129E77EF7804A2E713D8FB540FFED394095005EE2430800574F62E2441FD90CD
:2083C0000BA0E0FBA3E0FAA3E02402F9E43AFAED129E77EF540FFED394095005EE243080F5
:2083E0000574F62E2441FF900BA0E0FBA3E0FAA3E02403F9E43AFAEF129E77900BA0E0FB02
:20840000A3E0FAA3E02404F9E43AFAE4029E77900003E0FD75F002A42412F582E5F0340AED
:20842000F583E0FE75F002EDA42411F582E5F0340AF583E0FDEDFF900004E06EF0A3E06F2A
:20844000F0AFF9EFFEADFAEDFF900004E06EF0A3E06FF0900003E004F0E0D394054002E477
:20846000F09008867490F0E490087CF0A37420F0900004E0FCA3E090087EF0ECA3F09008DB
:20848000A0741DF0A37401F0A37408F0A3747CF0A37404F07B017A0879867D01028F92C0B8
:2084A000E0C0F0C083C082C0D075D000C000C001C002C003C004C005C006C0077F0C129B7E
:2084C0003F8F0D7F0C129B3F8F13750C00E50D4513543FF512E50D54C0FF6006E513F45F8D
:2084E000421285120DE51230E51F7F1C129B3F8F0CE50C541FC394124003430C80E50C5413
:208500001FD394065003430C40E50CFEE512420FEE420ED007D006D005D004D003D002D0AD
:2085200001D000D0D0D082D083D0F0D0E0327BFF7AA87984123000124800900869EFF070FE
:208540003E126926900822E07002A3E070089008697409F0802990086D7401F0A3740AF0A3
:20856000A3740AF0900A0EE0900870F0900858E0FBA3E0FAA3E0F91256C5900869EFF01287
:208580009BE1900957743EF0A37404F0900869E0900959F0900A5EE0FBA3E0FAA3E0240107
:2085A000F9E43AFA129E3C900A5DF0A37401F0A37409F0A37457F00298BC900B32E06404F6
:2085C0007061900B36E0FF605A64016056900B38E07050900B3AE0704A900B3CE07044A355
:2085E000E06002803E900B36E064027036900B39E07030900B3BE0FF64816005EF640270A6
:2086000022EFB48121E59620E7FB75960E759701E59620E7FB759611759710900B43740346
:20862000F080031217E3E59620E7FB75960EE4F597900B42E06404600BE59620E7FB75969D
:208640001175974822900894EFF0E4900896F0FF129744900895EFF0900894E0900AD1F027
:20866000601F900895E020E066D2B07FC87E00129C66900895E04401F0FDE4FF129916804A
:2086800041900895E0FF30E046EF54FE900895F0FDE4FF1299169008977401F0A374F4F0A9
:2086A00090089774FFF5F0129F3C45F060127F0E129744EF30E2097F017E001287DF80E045
:2086C000C2B0900894E060077F017E001287DF22900B32E064026025900B36E0701F900BAA
:2086E0003AE07019A3E07015A3E07011A3E0700D900B38E07007A3E0D3940140051217E365
:208700008044900B39E0D394004031900B327404F0E4900B43F0E59620E7FB75960E759780
:2087200001E59620E7FB759612759704E59620E7FB75960EE4F5971257FA800A900B32745A
:2087400003F0900B43F0900B42E06404600BE59620E7FB75961175974822900B32E06404A4
:20876000705B900B36E0FF605464016050900B38E0704A900B3AE07044900B3CE0703EA3D7
:20878000E060028038900B36E064027030900B39E0702A900B3BE0FF64817021EFB481206B
:2087A000E59620E7FB75960E759701E59620E7FB759611759740E4900B43F080031217E3F0
:2087C000E59620E7FB75960EE4F597900B42E06404600BE59620E7FB759611759748229064
:2087E00008AFEEF0A3EFF09008AF74FFF5F0129F3C45F060097FE87E03129C6680E922228F
:20880000900A0AE0FF900869F064126014E0FE6414600EEE64156009EE64166004EEB417E1
:20882000117B017A0A790B9008B77403F0128DAE801E900869E0C39480500D900A0AE0FF6A
:20884000A3E0FD1299168008900869E0FF129A75900957741BF0A37403F0E4A3F0900A5E66
:20886000E0FBA3E0FAA3E02401F9E43AFA129E3C900A5DF0A37401F0A37409F0A37457F09E
:208880000298BC900B36E06480701C900B38E07016A3E07012A3E0700EA3E0700AA3E07032
:2088A00006A3E0640160051217E38038900B32E0FFB40416900B3374FFF0A374B1F0A37427
:2088C00086F0900B40E4F0A304F0EFB40316900B3374FFF0A374B1F0A37488F0900B40E4E9
:2088E000F0A304F0900B42E064046018E59620E7FB759611759740900B427401F0E4900BAE
:208900003EF0A3F022C0E0C083C082C0D075D000C000C001C002C003C006C0077821E66008
:2089200051C2CF08860308E6FA08E62401F9E43AFA74FF129E55FF7822860308E6FA08E648
:20894000F9129E3CFEA807088002C313D8FCFF7822860308E6FA08E62401F9E43AFA129E73
:208960003C700B740226F618E436F6782116EF139293D007D006D003D002D001D000D0D01D
:20898000D082D083D0E032900894EFF07F02129744900B08E05403FEEF54FC4EFD7F0212E2
:2089A00099167F8F129A75750898E47830F6900B07E03333335418FF900B0BE0C4335420CB
:2089C0004FFF900B09E025E025E054044FF6900894E025E0541EFF900B08E0FEC43333549D
:2089E000C04F08F69008A0741FF0A3E4F0A37400F0A37430F0A37402F07B007A0079087DFE
:208A000001028F927F0A1297449008A3EFF07D227F011299169008A3E0FD7F0A1299167BE5
:208A2000017A0879A47D037F151293EE9008A5E054BFF07B017A0879A49008B77403F07F7F
:208A400015128DAEE4FD7F0D129916E4FF1297449008A3EFF0E4FF1297767F8F129A757FEC
:208A600097129A759008A3E04443F0FDE4FF129916C292D2937F017E001287DFC2A8029DD3
:208A80001E90086974FDF0124800900869EFF07029900A12E0FD90086E7401F0A3740AF07E
:208AA000A37414F0900A13E0900871F07B017A0A790A12538C900869EFF0129BE190095743
:208AC0007448F0A37403F0900869E0FF3395E0FE7CFF7DFF129E89900959EFF07B017A095A
:208AE0007957900A5EEBF0A3EAF0A3E9F02401F9E43AFA129E3C900A5DF00298BC900B934D
:208B0000EBF0A3EAF0A3E9F0129CCC900B97EFF0900B967433F0C2A89008BCE4F0A3F0A366
:208B2000F0A3F0A3F0A304F0FB7A0B7996FD128BEC9008BCE4F0A3F0A3F0A3F0A3F0A3F06C
:208B40007B017A0B79977D01128BEC900B93E0FBA3E0FAA3E02401F9E43AFA9008BCE4F096
:208B6000A3F0A3F0A3F0A37402F0E4A3F07DFB128BECD2A8227B017A0A790C90087CEBF0AB
:208B8000A3EAF0A3E9F0E4FF129E3C703B90087CE0FBA3E0FAA3E02401F9E43AFA129E3C51
:208BA000702690087CA3E0FAA3E02402F9E43AFA129E3C701390087CA3E0FAA3E02403F931
:208BC000E43AFA129E3C602390087CE0F9A3E0FAA3E0900882C9F0A3EAF0A3E9F090085865
:208BE000E0FBA3E0FAA3E0F9125DFB229008B8EBF0A3EAF0A3E9F09008C1E06002C294E41C
:208C0000FFEFC39D50259008B8E0FBA3E0FAA3E02FF9E43AFA129E3CF5A3E5F830E7FB753E
:208C2000F8019008C2E5A3F00F80D6E4FF9008BFE0FEEFC39E5022E4F5A3E5F830E7FB754A
:208C4000F8019008BCE0FBA3E0FAA3E02FF9E43AFAE5A3129E770F80D49008C0E06002D22E
:208C600094229008A6EFF0A3EBF0A3EAF0A3E9F0A3745EF0C2A89008BC7401F0A37408F013
:208C8000A374AAF0A37401F0E4A3F0A304F0FB7A0879AAFD128BEC9008AA747FF09008A783
:208CA000E0F9A3E0FAA3E09008BCC9F0A3EAF0A3E9F09008A6E09008BFF0A37402F0E4A3E0
:208CC000F07B017A0879AA7D01128BECD2A822900B32E064047024900B36E06481701C9085
:208CE0000B38E07016A3E07012A3E0700EA3E0700AA3E07006A3E0640160051217E38016E0
:208D0000900B3374FFF0A374B1F0A37488F0900B40E4F0A304F0900B42E064046018E5967D
:208D200020E7FB759611759740900B427401F0E4900B3EF0A3F02290088CEFF0D2937F013D
:208D40007E001287DF12797190088DEFF03395E0FEEF25E0FFEE33FE746D2FF9740A3EFAA6
:208D60007B0190088CE0FD124E0690088DE02FF07B017A08798C7D017C001281C3AD07AC39
:208D80000690088D12906090088DE02FF07B017A0A796DE0FD3395E0FC1298E7D29322F013
:208DA0007A0879A87B019008B77403F07F149008B3EFF0A3EBF0A3EAF0A3E9F09008B3E07F
:208DC0004420F0C2A89008BCE4F0A3F0A3F0A3F0A3F0A304F0FB7A0879B3FD128BEC900803
:208DE000B7E0FD9008BCE4F0A3F0A3F0A3F0A37402F0E4A3F09008B4E0FBA3E0FAA3E0F95E
:208E0000128BECD2A8229008707401F0A37401F0A3741AF0E4FFFEFD8047E47F087E07FD05
:208E2000FC90086CE0F8A3E0F9A3E0FAA3E0FBC312A0CF5035900870E0FBA3E475F0011238
:208E40009F3CA9F0FAE4129E7790086CE0FCA3E0FDA3E0FEA3E02401FFE43EFEE43DFDE4EF
:208E60003CFC90086C12A10680B022900894EBF0A3EAF0A3E9F0E4A3F07F80FE1298317FDD
:208E80008F129A757F5F7E00129831E50F20E023E50F541E600890089774FFF08026900836
:208EA00094E0FBA3E0FAA3E0F9124000900897EFF08011900894E0FBA3E0FAA3E0F9E4F580
:208EC000F0129F7D7F8F129A75900897E0FF22E4900869F07F0512974490086A129740EFF5
:208EE00030E211900869E024B8F0EF30E020E02405F0801A900869E024BEF0EF30E004E05A
:208F00002408F0EF30E107900869E024F6F0EFC41313540375F003A4FF90086AE090086925
:208F200030E706E0C39FF08003E02FF0900869E0FF22E0FBA3E0FAA3E0F99008C7EFF090BC
:208F400008CAEBF0A3EAF0A3E9F09008C8ECF0A3EDF04C603C9008C7E0F5964396C0E4FF81
:208F6000FED39008C9E09F9008C8E09E4020E59620E7FB9008CAE0FBA3E0FAA3E02FF9EA36
:208F80003EFAE597129E770FBF00010E80D3E4F596229008A0E04420F0C2A89008BCE4F037
:208FA000A3F0A3F0A3F0A3F0A304F0128BEC9008BCE4F0A3F0A3F0A3F0A3F0A3F07B017A48
:208FC0000879A07D01128BEC9008A4E0FD9008BCE4F0A3F0A3F0A3F0A37402F0E4A3F0905F
:208FE00008A1E0FBA3E0FAA3E0F9128BECD2A822E4FFFE0FBF00010EBE01F8BFF4F522226E
:20900000900A5CE0703204F09008CAF0A3740AF0A37408F0900A49E0FBA3E0FAA3E024018F
:20902000F9E43AFA129E3C049008CDF0900A49A3E0FAA3E0F9023FBF900A49E0FBA3E0FAC3
:20904000A3E0F9129E3C9008CAF0900A08E09008CBF07BFF7AA879BF12300022AD07AC06E3
:20906000E0FF3395E0FEEF25E0FFEE33FE746D2FF9740A3EFA7B019008A3EBF0A3EAF0A3E8
:20908000E9F0A3ECF0A3EDF0F4FFECF4FE9008A6F0A3EFF0EEFD124E069008A4E475F0049D
:2090A000129F269008A3E0FBA3E0FAA3E0F9A3A3E0FD124E067F0422900B7DEFF0900B808A
:2090C000EBF0A3EAF0A3E9F0900B7EECF0A3EDF04C603BE59620E7FB900B7DE0F596E4FF7D
:2090E000FED3900B7FE09F900B7EE09E4020900B80E0FBA3E0FAA3E02FF9EA3EFA129E3CE3
:20910000F597E59620E7FB0FBF00010E80D3229008C7EFF09008CAEBF0A3EAF0A3E9F090F0
:2091200008C8ECF0A3EDF04C603BE59620E7FB9008C7E0F596E4FFFED39008C9E09F9008A9
:20914000C8E09E40209008CAE0FBA3E0FAA3E02FF9EA3EFA129E3CF597E59620E7FB0FBF1F
:2091600000010E80D322C0E0C083C082C0D075D000C000C001C002C003C2997916E778150D
:20918000667005781BF680187817860308E6FA08E6F97816E60629F9E43AFA129E3CF599BE
:2091A00030980678147601C298D003D002D001D000D0D0D082D083D0E03290089CEEF0A362
:2091C000EFF0A3ECF0A3EDF090089CE0550EFEA3E0550F4E7024A3E07002A3E0601CE59109
:2091E00030E7E57FE87E031297DB90089FE024FFF090089EE034FFF080CE90089EE07002CE
:20920000A3E07009129C2D750E00750F0122900B36E0701D900B3AE07017A3E07013A3E04A
:20922000700FA3E0700B900B38E07005A3E030E7031217E3900B427405F0900B39E0900B4B
:209240003260057403F080037402F0900B42E06404600BE59620E7FB7596117597482290F8
:209260000A0AE0600EA3E0B4FF047F018002E4FF128645900A0DE06006A3E0FF126C77909C
:2092800009577419F0A3740EF0E4A3F0A3F0A3F0A3F0128ECF90095DEFF0900A5D740EF0FF
:2092A000A37401F0A37409F0A37457F00298BC127FFAEF603CE490085CF0900A08E0645DC1
:2092C0006003125F61900A08E075F003A42486F582E5F034ACF583E4740193FA740293F995
:2092E00012A158900854E07003129CC6E4900854F090085CE060057F01129BCF2274022FF4
:20930000F58274093EF583E0FF9009A3E0600BE4F09009A2F0781BE670FB9009A2E024A477
:20932000F582E43409F583EFF09009A2E004F0E0FDC394645004EFB40A0F7B017A0979A46B
:209340001297AA9009A37401F0229008C7EFF0E4A3F09008C8E0FFD394035039EF25E025F7
:20936000E02461F582E4340AF583E0FF9008C7E0FEEFB50618A3E025E025E02462F582E42B
:20938000340AF583A3E0FAA3E0F902A1589008C8E004F080BD22900A09E064047043900959
:2093A000577456F0A37403F07B017A097957900A5EEBF0A3EAF0A3E9F02401F9E43AFA12AF
:2093C0009E3C900A5DF09009597401F01298BC7F647E001287DFE4FDFF7E1012986275EF58
:2093E0001022EFF07A08797E7B017D037F149008B3EFF0A3EBF0A3EAF0A3E9F0C2A89008B1
:20940000B3E04460F0A3E0F9A3E0FAA3E09008BCC9F0A3EAF0A3E9F0A3EDF0A37402F0A377
:2094200014F0FB7A0879B3FD128BECD2A822E59620E7FB759601759708E59620E7FB759638
:2094400007759707E59620E7FB759609759707E59620E7FB75960B75970775D7E0E59620E1
:20946000E7FB75960F75978043E602D2AFE59620E7FB75960175970122900B39E0FF1293A8
:209480004A900A5EE0F9A3E0FAA3E0900B33C9F0A3EAF0A3E9F0900A5DE0FF900B40E4F0AC
:2094A000A3EFF0900B42E064046018E59620E7FB759611759740900B427401F0E4900B3EA9
:2094C000F0A3F022E4F50EF50F7D03FF129916C292D293129D217B017A0879B07D037F15F8
:2094E0001293EE9008B1E04440F07B017A0879B09008B77403F07F15128DAE7F0C12974406
:20950000E4F50EF50F7D3F7F0D129916D2A82212102F900A49E0F9A3E0FAA3E0900B33C917
:20952000F0A3EAF0A3E9F0900B3CE0FFA3E0900B40CFF0A3EFF0900B42E064046018E596D5
:2095400020E7FB759611759740900B427402F0E4900B3EF0A3F02290086BEFF090085BE047
:20956000FE6F6031EE24FE60080470081267FF8003129D1890086BE024FE600E04700E7BC7
:20958000017A08794F129D1B8003129CB790086BE090085BF022E4900869F0129BE19009EA
:2095A00057744CF0A37440F0900869E0900959F0A3740AF07B017A097957900A5EEBF0A344
:2095C000EAF0A3E9F02401F9E43AFA129E3C900A5DF00298BCE4900869F0129BE190095783
:2095E0007450F0A37440F0900869E0900959F0A3740AF07B017A097957900A5EEBF0A3EA6D
:20960000F0A3E9F02401F9E43AFA129E3C900A5DF00298BCD2937F067E001287DF90088285
:2096200074AAF0900884F0900886740AF09008837408F0900885F09008877404F07B017A73
:209640000879827D037C001298E7D2937F017E000287DFE47814F6781BF67815F608F690AF
:2096600009A3F09009A2F0C29FD29DD29C758840758920438E08758D30D28E43A41075E1D2
:209680000175B283D2BC75A890D2ACD2AF43E24022900B36E06401701C900B3CE07016A3DC
:2096A000E07012900B38E0700CA3E07008A3E07004A3E060031217E3900B42E06404600BA5
:2096C000E59620E7FB7596117597482274FF900869F0A3F0EE3395E0FDFCE47B30FAF9F87B
:2096E000129F9CC374FF9F90086AF074FF9E900869F0E4F5C8438E30E0FEA3E0FDF5CA8D08
:20970000CCEEF5CBF5CD2243A40443A701D282C2B075A16075A20B75F801129C4643A40569
:2097200043A60675A51FD2A043E10243E2C0C290D291D294C2A17F647E00129C66D2A122FC
:20974000EFF07F0A9008B3EFF0C2A8E04440F09008BC7401F0A37408F0A374B4F0A374011E
:20976000F0A3F0A3F0FB7A0879B3FD128BECD2A89008B4E0FF229008A7EFF070077D407F0C
:20978000091299169008A7E0B406077D807F091299167F03129744EF540FFF9008A7E0FEFC
:2097A000C454F04FFD7F03029916E490090FF0781BE670FB781B76017817A60308A60208C8
:2097C000A60178167601AF0518A6077817860308E6FA08E6F9129E3CF599227C007D0412D2
:2097E000A15EC374FF9FFF74FF9EFC538EBFE4F591EFFBF592ECF5938B94F59543910422F7
:209800007E007F407D007B017A09795712A335900957745CF0A37440F0E4A3F0900A5D74FC
:2098200040F0A37401F0A37409F0A37457F00298BC8E108F11E4FFFEE50E5510FCE50F5570
:20984000114C700B0FBF00010EBEFFECBFFDE9D3EF94F0EE94FF4009129C2D750E00750F13
:209860000122A2AF9201C2AF75FF8075EF028E108F1175B7A575B7F1438F0175FF8075EFBF
:2098800002851182851083EDF0538FFEA20192AF229009577405F0900955E0900958F0903B
:2098A0000956E0900959F0900A5E7401F0A37409F0A37457F0900A5D7403F022E490087C44
:2098C000F0900958E0FF90087CE0FEC39F501774572EF582E43409F583E0FF129C3A9008A5
:2098E0007CE004F080DB227822A60308A60208A601E408F6AF057821A60775C804AFA87510
:20990000A820D2AF7821E670FB30CFFD8FA8E4F5C822E0FDE4FF9008B3EFF0A3EDF0C2A84A
:209920009008BCE4F0A3F0A3F0A3F0A304F0A3F0FB7A0879B37D02128BECD2A822129968BC
:20994000EF3395E0FEEF2480FFE43EAB07FA7C007D0CFE129E89AC06AD07EAC313FEEB13B4
:209960002DFBEC3EFEAF03227F87129A757F147E00129C667F19129744EF5480FD3395E08A
:209980004D6006EF547FFE8006EF547FF404FEAF0622900B9DEBF0A3EAF0A3E9F0900B9DFB
:2099A000E0FBA3E0FAA3E0F912A901AD07900B9DE0FBA3E0FAA3E0F90297AA90084BE070E1
:2099C00002A3E070037F0122129BA9C390084CE09F90084BE09E500990084E7401F07F00ED
:2099E000227F01227F96129A757F97129A757FF47E01129C667F0F129744900892EFF07F2D
:209A000096129A75900892E0FF22438E045388EF53D8BFE58954F04401F589E4F58AF58C82
:209A200075D90475D840F5F9F5FA43881022C2948FA3E5F830E7FB75F801E5A3129E77E4F5
:209A4000F5A3E5F830E7FB75F801E5A3129E77D294229009597402F09009577415F0A37402
:209A600003F0900A5DF0A37401F0A37409F0A37457F00298BC9008A7EFF0C2A89008BCE480
:209A8000F0A3F0A3F0A3F0A304F0A3F0FB7A0879A7FD128BECD2A822900BA6EFF0A3EDF094
:209AA0009008BCE4F0A3F0A3F0A3F0A3F0A304F0FB7A0B79A67D02028BEC43B203E4F5B97A
:209AC00043B980128FF043B9C0128FF0E5B930E5FB75B69075A90322E4FF129744EF30E7AA
:209AE00013EF547FFDE4FF1299167F017E001287DF1270002275F003EFA42486F582E5F0E5
:209B000034ACF583740193FA740293F902A158900A49E0FBA3E0FAA3E02401F9E43AFA12E8
:209B20009E3C9009A0F022C2A89008BCE4F0A3F0A3F0A3F0A304F0A3F0128BECD2A822C2A4
:209B4000A8EF4440FF7B017A097910129A2ED2A8900910E0FF22EF30E7028009EF547FFF13
:209B6000C3747F9FFFAD077F180299167F18129744EF30E7028009EF547FFFC3747F9FFF6B
:209B800022900B42E06404600BE59620E7FB75961175974822900AD2E0FD7F0512991690E6
:209BA0000AD3E0FD7F0A029916AFFA7E00ADF97C00ABFAEBB507F2EFFEEDFF22E4FF1297A3
:209BC00044EF20E709EF4480FDE4FF12991622124C181298BC7F02900959E06003B401EF96
:209BE00022129A0AE4FF12864590085CE07003127A27229008C7E004F070069008C6E004C6
:209C0000F0229008C7E004F070069008C6E004F0229001197401F0900A0AE0FF029BCFE453
:209C200090085BF0A3F0900854F0027A27127A277F017E001287DF025F61781BE670FB78E8
:209C40001B76018F9922D28375E40BD288D2A8D2AF227814E670FBE47814F6227F0D7E0089
:209C60001296CC7F00221297DBE59130E7FB227F02129557026F7C7F02129557028A817F2A
:209C8000011295570268007F0112955702739C7F011295570265107F0112955702663F7F33
:209CA0000112955702852E7F011295570246E37F011295570263DFE4FF1297767F0022E4FE
:209CC0007814F6AF9922E4900A5CF0227F1312974422E47814F6227F15028D377F0A028D11
:209CE000377F09028D377F08028D377F02028C627F9D029A757F80029A757F01227F0022A1
:209D0000025FFF0276A402925F02880002812E027CEB0282587F00227F00220244B4C294C2
:209D200022D29422E709F608DFFA8046E709F208DFFA803E88828C83E709F0A3DFFA803244
:209D4000E309F608DFFA8078E309F208DFFA807088828C83E309F0A3DFFA806489828A832C
:209D6000E0A3F608DFFA805889828A83E0A3F208DFFA804C80D280FA80C680D4806980F2B6
:209D80008033801080A680EA809A80A880DA80E280CA803389828A83ECFAE493A3C8C582CE
:209DA000C8CCC583CCF0A3C8C582C8CCC583CCDFE9DEE7800D89828A83E493A3F608DFF98F
:209DC000ECFAA9F0EDFB2289828A83ECFAE0A3C8C582C8CCC583CCF0A3C8C582C8CCC58344
:209DE000CCDFEADEE880DB89828A83E493A3F208DFF980CC88F0EF60010E4E60C388F0EDB1
:209E00002402B4040050B9F582EB2402B4040050AF2323458223909D7473C2D530F707B261
:209E2000D563F0FF05F030E70CB2D5F4048463F0FF05F080018430D502F40422BB01068928
:209E4000828A83E0225002E722BBFE02E32289828A83E49322BB010989828A83F8E028F0D8
:209E600022500327F722BBFE05F8E328F3228A838982F8E4932822BB010689828A83F0229A
:209E80005002F722BBFE01F322EF8DF0A4A8F0CF8CF0A428CE8DF0A42EFE22BC000BBE0007
:209EA00029EF8DF084FFADF022E4CCF875F008EF2FFFEE33FEEC33FCEE9DEC984005FCEE21
:209EC0009DFE0FD5F0E9E4CEFD22EDF8F5F0EE8420D21CFEADF075F008EF2FFFED33FD408D
:209EE00007985006D5F0F222C398FD0FD5F0EA22C2D5EC30E709B2D5E4C39DFDE49CFCEE87
:209F000030E715B2D5E4C39FFFE49EFE129E9BC3E49DFDE49CFC8003129E9B30D507C3E440
:209F20009FFFE49EFE22C5F0F8A3E028F0C5F0F8E582158270021583E038F022A3F8E0C57A
:209F4000F025F0F0E582158270021583E0C838F0E822BB010A89828A83E0F5F0A3E0225092
:209F60000687F009E71922BBFE07E3F5F009E3192289828A83E493F5F074019322BB010A26
:209F800089828A83F0E5F0A3F0225006F709A7F01922BBFE06F3E5F009F31922E88FF0A43E
:209FA000CC8BF0A42CFCE98EF0A42CFC8AF0EDA42CFCEA8EF0A4CDA8F08BF0A42DCC382542
:209FC000F0FDE98FF0A42CCD35F0FCEB8EF0A4FEA9F0EB8FF0A4CFC5F02ECD39FEE43CFCEA
:209FE000EAA42DCE35F0FDE43CFC2275F008758200EF2FFFEE33FECD33CDCC33CCC58233C6
:20A00000C5829BED9AEC99E58298400CF582EE9BFEED9AFDEC99FC0FD5F0D6E4CEFBE4CDFC
:20A02000FAE4CCF9A88222B800C1B90059BA002DEC8BF084CFCECDFCE5F0CBF97818EF2F27
:20A04000FFEE33FEED33FDEC33FCEB33FB10D703994004EB99FB0FD8E5E4F9FA227818EF07
:20A060002FFFEE33FEED33FDEC33FCC933C910D7059BE99A4007EC9BFCE99AF90FD8E0E49B
:20A08000C9FAE4CCFB2275F010EF2FFFEE33FEED33FDCC33CCC833C810D7079BEC9AE89944
:20A0A000400AED9BFDEC9AFCE899F80FD5F0DAE4CDFBE4CCFAE4C8F922EB9FF5F0EA9E42D2
:20A0C000F0E99D42F0EC6480C864809845F022EB9FF5F0EA9E42F0E99D42F0E89C45F022B1
:20A0E000E8600FECC313FCED13FDEE13FEEF13FFD8F122E8600FEFC333FFEE33FEED33FDEC
:20A10000EC33FCD8F122ECF0A3EDF0A3EEF0A3EFF022BB010789828A8302A36A5005E9F898
:20A1200002A361BBFE05E9F802A37389828A8302A37CD083D082F8E4937012740193700D0E
:20A14000A3A393F8740193F5828883E4737402936860EFA3A3A380DF8A838982E473EC8E5C
:20A16000F0A4CCC5F0CCCDF8EFA4CEC5F02DFDE43CFCE8A42EC8C5F03DFDE43CFCEFA4FFBE
:20A18000E5F028FEE43DFDE43CFC22E3F5F009E208B5F06BDFF58067E3F5F009E608B5F07E
:20A1A0005EDFF5805A87F009E608B5F052DFF6804E87F009E208B5F046DFF6804288828C09
:20A1C0008387F009E0A3B5F036DFF6803288828C8387F009E493A3B5F025DFF5802188829B
:20A1E0008C83E3F5F009E0A3B5F014DFF5801088828C83E3F5F009E493A3B5F002DFF4025F
:20A20000A2BA808780E9809080D4803E8015806E807E809D80B7808D80A380518074803CCA
:20A2200002A2C689828A83ECFAE493F5F0A3C8C582C8CCC583CCE493A3C8C582C8CCC583FB
:20A24000CCB5F076DFE3DEE1807089828A83E493F5F0A3E208B5F062DFF4805E89828A83D5
:20A26000E0F5F0A3E608B5F051DFF5804D89828A83E0F5F0A3E208B5F040DFF5803C898207
:20A280008A83E493F5F0A3E608B5F02EDFF4802A8002805789828A83ECFAE493F5F0A3C856
:20A2A000C582C8CCC583CCE0A3C8C582C8CCC583CCB5F006DFE4DEE280007FFFB5F0020F93
:20A2C0002240027F012289828A83ECFAE0F5F0A3C8C582C8CCC583CCE0A3C8C582C8CCC570
:20A2E00083CCB5F0D5DFE5DEE380CF89828A83ECFAE0F5F0A3C8C582C8CCC583CCE493A38A
:20A30000C8C582C8CCC583CCB5F0AFDFE4DEE280A988F0EF60010E4E60ABED2402B404008C
:20A320005098F582EB2402B40400508E232345822390A20273EF4E6012EF60010EEDBB018A
:20A340000B89828A83F0A3DFFCDEFA2289F05007F709DFFCA9F022BBFEFCF309DFFCA9F0E7
:20A3600022E6FB08E6FA08E6F922E0FBA3E0FAA3E0F922E2FB08E2FA08E2F922E493FB7447
:20A380000193FA740293F9227265616420726567733A202568687820256868782025686835
:20A3A0007820256868780A00454E2070696E206661696C65640A004952512070696E202F63
:20A3C0002072656164696E672049525120666C616773206661696C65640A0043616E6E6FCC
:20A3E000742072756E206F6E204153333939300A0043616E6E6F742072756E206F6E2041AE
:20A4000053333939310A00556E6B6E6F776E206368697020256868780A000A726567202531
:20A4200068687820202000256868782000256868780000000102030405060708090A0B0C2C
:20A440000D0E0F101112131415161718191A1B1C1D1E1F202122232425262728292A2B2C6C
:20A460002D2E2F303132333435363738393A3B3C3D3E3F404142434445464748494A4B4C4C
:20A480004D4E4F505152535455565758595A5B5C5D5E5F606162636465666768696A6B6C2C
:20A4A0006D6E6F707172737475767778797A7B7C7D7E7F808182838485868788898A8B8C0C
:20A4C0008D8E8F909192939495969798999A9B9C9D9E9FA0A1A2A3A4A5A6A7A8A9AAABACEC
:20A4E000ADAEAFB0B1B2B3B4B5B6B7B8B9BABBBCBDBEBFC0C1C2C3C4C5C6C7C8C9CACBCCCC
:20A50000CDCECFD0D1D2D3D4D5D6D7D8D9DADBDCDDDEDFE0E1E2E3E4E5E6E7E8E9EAEBECAB
:20A52000EDEEEFF0F1F2F3F4F5F6F7F8F9FA011A00011400011B01500B57BFAFA7A3A1A0D2
:20A54000B0B8BCBE41888A642082490B455580C0E0F0F8FCFEFF490B4EFF7F3F1F0F07033A
:20A560000100480998FFFFFFFFFFFFFFFF604009150000000000000000000000000000003B
:20A580000000000000000000000000000000000000000000000000000000000000000000BB
:20A5A0000000000000000000000000000000000000490B67FFAC65FFAC6AFFAC76430B420A
:20A5C0000003034C0A6105FF98910000000000000000500A4C02FF9B0F0000000000000040
:20A5E0000000000000410A5C0045084F0C0200000141085704410862034108613244085D32
:20A60000000DC65E44000B000E261242084600004208240190420855000041085C00410858
:20A620004D0241000000410001004100020041000300420B0C000A010D00010C00020E0033
:20A6400000410AD100420AEFBB80410AF10000666F756E64207769746820706F77536C6F90
:20A66000743D2568687820257820746167732C206D617820256868780A002D002E00202567
:20A680006868780A002048656C6C6F20576F726C64210A204D79206E616D65206973204DF1
:20A6A0004952434F210A2057656C636F6D6520746F20766973697420726669642E656C65DB
:20A6C000636B6974732E636F6D0A00617333393978496E697469616C697A6528292072659A
:20A6E0007475726E65642025780A005072696E74205043202568687820256868780A0050CD
:20A7000072696E742045504320002568687820000A0054414720256868783A0A00524E314F
:20A72000363A202568687820256868780A004E756D626572206F66207265616420627974FC
:20A7400065733A2025640A0050433A20256868782025686878004550433A20004550434CF7
:20A76000454E20286279746573293A20256868640A0048414E444C453A2025686878202539
:20A780006868780A000000787FE4F6D8FD75817F75D90002A7D1022000E493A3F8E493A336
:20A7A0004003F68001F208DFF48029E493A3F85407240CC8C333C4540F4420C8834004F400
:20A7C00056800146F6DFE4800B010204081020408090A52EE47E019360BCA3FF543F30E55A
:20A7E00009541FFEE493A360010ECF54C025E060A840B8E493A3FAE493A3F8E493A3C8C5A1
:20A8000082C8CAC583CAF0A3C8C582C8CAC583CADFE9DEE780BE63617574696F6E20777205
:20A820006F6E6720636869700A0041533339393220526561646572204669726D77617265CB
:20A8400020322E322E390A0041533339393220456C65636B69747320436F6C7420616E6411
:20A86000204D4943524F20312E320A0057726F6E672076657273696F6E20747970652073DB
:20A88000656E64004B494C4C205461670A0025686878202568687820256868782025686873
:20A8A0007820256868782025686878202568687820256868780A002568687820000A0075D6
:20A8C0007362206572726F72202D207265706F72742025686878206C6F7374206166746521
:20A8E0007220256868780A000A0A53656E645061636B65742074696D6564206F75740A0A9A
:20A9000000E4FFFE129E3C600C0FEF70010E09E970F20A80EF2212011001000000402513F6
:20A9200029C00000010200010902290001010080AF09040000020300000009210101000186
:20A9400022140307058103400001070502034000010600FF0901A10185109502750826FF1C
:20A960000015000901910285119530750826FF0015000901810285319502750826FF001582
:20A9800000090191028532953F750826FF001500090181028533953F750826FF00150009FF
:20A9A00001910285349502750826FF001500090181028514953D750826FF001500090191B2
:20A9C0000285159502750826FF001500090181028518950D750826FF0015000901910285E8
:20A9E00019950D750826FF001500090181028535953F750826FF0015000901910285369526
:20AA000003750826FF0015000901810285379507750826FF001500090191028538953F753D
:20AA20000826FF00150009018102851C9502750826FF00150009019102851D9505750826DC
:20AA4000FF00150009018102851A9505750826FF00150009019102851B9502750826FF00EF
:20AA6000150009018102853F950C750826FF001500090191028540950F750826FF0015005B
:20AA8000090181028547953F750826FF0015000901910285489502750826FF001500090110
:20AAA00081028549950C750826FF00150009019102854A953F750826FF0015000901810269
:20AAC000854B953F750826FF00150009019102854C953F750826FF00150009018102854DC3
:20AAE000953F750826FF00150009019102854E953F750826FF00150009018102854F953F9B
:20AB0000750826FF001500090191028550953F750826FF001500090181028541953F7508DD
:20AB200026FF001500090191028542953F750826FF0015000901810285439502750826FF5E
:20AB4000001500090191028544953F750826FF00150009018102853B9507750826FF00154F
:20AB60000009019102853E9502750826FF00150009018102853D9506750826FF001500097D
:20AB8000019102853C9502750826FF0015000901810285459509750826FF001500090191CB
:20ABA0000285469504750826FF001500090181028555953F750826FF001500090191028564
:20ABC000569502750826FF001500090181028558953F750826FF00150009018102855795DE
:20ABE00001750826FF00150009019102855A953F750826FF001500090181028559953F75E2
:20AC00000826FF00150009019102855C953F750826FF00150009018102855B953F75082605
:20AC2000FF00150009019102855E953F750826FF00150009018102855D9503750826FF004C
:20AC40001500090191028560953F750826FF00150009018102855F953F750826FF001500D6
:20AC600009019102C005030904000A0361006D007300200000000E034100530033003900E3
:20AC8000390078000000FF9D00FF9D00FF9D00FF9D00FF9D00FF9D00FF9D00FF9D00FF9D87
:20ACA00000FF9D00FF9D00FF9D00FF9D00FF9D00FF9D00FF9D00FF9D03FF9D00FF9D00FF7A
:20ACC0009D00FF9A52FF9D00FF9D00FF9D00FF9D06FF9D00FF9D09FF9D00FF9D0CFF9D0055
:20ACE000FF9D00FF9D00FF9D00FF9D00FF9D00FF9D00FF9D00FF9D00FF9D00FF9D00FF9DA0
:20AD000000FF9D00FF9D00FF9D00FF9D00FF9D00FF9D00FF9D00FF9D00FF2FEAFF9D00FFA0
:20AD20009C7FFF9D00FF9C87FF9D00FF9C8FFF9D00FF9D00FF9D00FF9C97FF9D00FF9C9F98
:20AD4000FF9D00FF51CFFF9D00FF1800FF9D00FF9C11FF9D00FF9CA7FF9D00FF9C77FF9D15
:20AD600000FF9C6FFF9D00FF9596FF9D00FF7E47FF9D00FF95D5FF9D00FF9D00FF9D00FFCB
:20AD80009D00FF9D00FF9396FF9D00FF9D12FF9D00FF9D0FFF9D00FF9800FF9D00FF4FB9EB
:20ADA000FF9D00FF9CAFFF9D00FF9D00FF9D00FF9D00FF9D00FF9D00FF9D00FF9D00FF9D31
:20ADC00000FF9D00FF9D00FF9D00FF9D00FF9D00FF9D00FF9D00FF9D00FF9D00FF9D00FF5C
:20ADE0009D00FF9D00FF9D00FF9D00FF9D00FF9D00FF9D00FF9D00FF9D00FF9D00FF9D009E
:20AE0000FF9D00FF9D00FF9D00FF9D00FF9D00FF9D00FF9D00FF9D00FF9D00FF9D00FF9D7E
:20AE200000FF9D00FF9D00FF9D00FF9D00FF9D00FF9D00FF9D00FF9D00FF9D00FF9D00FFFB
:20AE40009D00FF9D00FF9D00FF9D00FF9D00FF9D00FF9D00FF9D00FF9D00FF9D00FF9D003D
:20AE6000FF9D00FF9D00FF9D00FF9D00FF9D00FF9D00FF9D00FF9D00FF9D00FF9D00FF9D1E
:20AE800000FF9D00FF9D00FF9D00FF9D00FF9D00FF9D00FF9D00FF9D00FF9D00FF9D00FF9B
:20AEA0009D00FF9D00FF9D00FF9D00FF9D00FF9D00FF9D00FF9D00FF9D00FF9D00FF9D00DD
:20AEC000FF9D00FF9D00FF9D00FF9D00FF9D00FF9D00FF9D00FF9D00FF9D00FF9D00FF9DBE
:20AEE00000FF9D00FF9D00FF9D00FF9D00FF9D00FF9D00FF9D00FF9D00FF9D00FF9D00FF3B
:20AF00009D00FF9D00FF9D00FF9D00FF9D00FF9D00FF9D00FF9D00FF9D00FF9D00FF9D007C
:20AF2000FF9D00FF9D00FF9D00FF9D00FF9D00FF9D00FF9D00FF9D00FF9D00FF9D00FF9D5D
:20AF400000FF9D00FF9D00FF9D00FF9D00FF9D00FF9D00FF9D00FF9D00FF9D00FF9D00FFDA
:20AF60009D00FF9D00FF9D00FF9D00FF9D00FF9D00FF9D00FF9D00FF9D00FF9D00FF9D001C
:20AF8000FF9D00FF9D000000102120423063408450A560C670E781089129A14AB16BC18C86
:20AFA000D1ADE1CEF1EF123102103273225252B5429472F762D693398318B37BA35AD3BD76
:20AFC000C39CF3FFE3DE246234430420140164E674C744A45485A56AB54B85289509E5EEB6
:20AFE000F5CFC5ACD58D365326721611063076D766F6569546B4B75BA77A97198738F7DF36
:20B00000E7FED79DC7BC48C458E5688678A70840186128023823C9CCD9EDE98EF9AF89486D
:20B020009969A90AB92B5AF54AD47AB76A961A710A503A332A12DBFDCBDCFBBFEB9E9B7975
:20B040008B58BB3BAB1A6CA67C874CE45CC52C223C030C601C41EDAEFD8FCDECDDCDAD2A35
:20B06000BD0B8D689D497E976EB65ED54EF43E132E321E510E70FF9FEFBEDFDDCFFCBF1B35
:20B08000AF3A9F598F78918881A9B1CAA1EBD10CC12DF14EE16F108000A130C220E35004AA
:20B0A00040257046606783B99398A3FBB3DAC33DD31CE37FF35E02B1129022F332D2423595
:20B0C000521462777256B5EAA5CB95A88589F56EE54FD52CC50D34E224C314A00481746695
:20B0E000644754244405A7DBB7FA879997B8E75FF77EC71DD73C26D336F2069116B0665755
:20B10000767646155634D94CC96DF90EE92F99C889E9B98AA9AB584448657806682718C04C
:20B1200008E1388228A3CB7DDB5CEB3FFB1E8BF99BD8ABBBBB9A4A755A546A377A160AF194
:20B140001AD02AB33A92FD2EED0FDD6CCD4DBDAAAD8B9DE88DC97C266C075C644C453CA214
:20B160002C831CE00CC1EF1FFF3ECF5DDF7CAF9BBFBA8FD99FF86E177E364E555E742E9354
:20B180003EB20ED11EF0010000000000FFFFFFFFFFFFFFFFFFFFFFFFFFFFFFFFFFFFFFFFE5
:20B1A000FFFFFFFFFFFFFFFFFFFFFFFFFFFFFFFFFFFFFFFFFFFFFFFFFFFFFFFFFFFFFFFFAF
:20B1C000FFFFFFFFFFFFFFFFFFFFFFFFFFFFFFFFFFFFFFFFFFFFFFFFFFFFFFFFFFFFFFFF8F
:20B1E000FFFFFFFFFFFFFFFFFFFFFFFFFFFFFFFFFFFFFFFFFFFFFFFFFFFFFFFFFFFFFFFF6F
:20B20000FFFFFFFFFFFFFFFFFFFFFFFFFFFFFFFFFFFFFFFFFFFFFFFFFFFFFFFFFFFFFFFF4E
:00000001FF
